:100000000C9446040C9458040C9458040C9401105D
:100010000C9437320C9458040C9458040C945804E3
:100020000C9458040C9458040C9458040C94932980
:100030000C9458040C9458040C9458040C945804D0
:100040000C94A72B0C9458040C942D250C94EF249D
:100050000C9458040C9458040C9458040C945804B0
:100060000C9458040C9458047607790F790F800784
:100070008D079A07A707790FAB07790FB907790F93
:10008000C307CD07FE07790F790F790FD707E4076C
:10009000F107420E530E720E530E760E890E7C0E31
:1000A000820E9E0EA40EB30ECA0EEE0EF80E040FB4
:1000B0000E0FD81FDB1FE01FE31FE61FE91FEC1F19
:1000C000EF1FF21FF51FF81F0720FB1F0720072057
:1000D00007200720072007200120FE1F04204E20B4
:1000E0005120542057205A205D2060206320A727EC
:1000F000AD27B027B327B827C027CA2748284828E4
:100100004828D227D527DE27E72748284828482827
:10011000482848284828EF27F92705280D281028BF
:100120001928222828284828482831283A28084A07
:10013000D73B3BCE016E84BCBFFDC12F3D6C7431FB
:100140009ABD56833DDA3D00C77F11BED9E4BB4C52
:100150003E916BAAAABE000000803F05A84CCDB21C
:10016000D44EB93836A9020C50B9918688083CA6FD
:10017000AAAA2ABE000000803F003E0D0A007C00B3
:10018000300031007C002C50696E3A002C52583AF5
:10019000002C4275663A002C002C57506F733A00C1
:1001A0002C002C4D506F733A003C446F6F72003C32
:1001B000436865636B003C416C61726D003C486F45
:1001C0006D65003C486F6C64003C52756E003C49A4
:1001D000646C65005D0D0A005B312E30632E323099
:1001E0003135313130393A000D0A003D00244E00DE
:1001F0005D0D0A00205300204600205400204D379A
:1002000000204D3800204D3900204D3500204D3460
:1002100000204D3300204D3200204D3100204D3064
:100220000020473934002047393300204739310056
:10023000204739300020473230002047323100203B
:1002400047313900204731380020473137002047F7
:10025000004733382E00473830004733004732001C
:100260004731004730005B005D0D0A005B544C4F86
:100270003A005D0D0A002C005B4739323A005D0DF3
:100280000A002C003A003330003238005B47005D32
:100290000D0A003A002C005B5052423A00290D0A28
:1002A00000206D61782074726176656C2C206D6D14
:1002B0000020616363656C2C206D6D2F7365635E38
:1002C0003200206D617820726174652C206D6D2F75
:1002D0006D696E002C20737465702F6D6D007A004F
:1002E000790078002028003D002400202872706DDD
:1002F000206D696E290D0A00202872706D206D61D5
:1003000078290D0A2433313D002028686F6D696E0D
:10031000672070756C6C2D6F66662C206D6D290DD5
:100320000A2433303D002028686F6D696E672064B1
:1003300065626F756E63652C206D736563290D0AA8
:100340002432373D002028686F6D696E6720736521
:10035000656B2C206D6D2F6D696E290D0A24323668
:100360003D002028686F6D696E6720666565642CA6
:10037000206D6D2F6D696E290D0A2432353D0029DF
:100380000D0A2432343D002028686F6D696E6720A5
:1003900064697220696E76657274206D61736B3A60
:1003A000002028686F6D696E67206379636C652C27
:1003B00020626F6F6C290D0A2432333D00202868BB
:1003C000617264206C696D6974732C20626F6F6C4C
:1003D000290D0A2432323D002028736F6674206C88
:1003E000696D6974732C20626F6F6C290D0A243259
:1003F000313D0020287265706F727420696E6368E9
:1004000065732C20626F6F6C290D0A2432303D0019
:10041000202861726320746F6C6572616E63652C55
:10042000206D6D290D0A2431333D0020286A756E38
:100430006374696F6E20646576696174696F6E2C90
:10044000206D6D290D0A2431323D00290D0A243119
:10045000313D002028737461747573207265706F6C
:100460007274206D61736B3A00202870726F626540
:100470002070696E20696E766572742C20626F6FD1
:100480006C290D0A2431303D0020286C696D697497
:100490002070696E7320696E766572742C20626FAD
:1004A0006F6C290D0A24363D002028737465702076
:1004B000656E61626C6520696E766572742C20626F
:1004C0006F6F6C290D0A24353D00290D0A24343D37
:1004D00000202864697220706F727420696E7665DE
:1004E0007274206D61736B3A00290D0A24333D004C
:1004F00020287374657020706F727420696E766541
:100500007274206D61736B3A0020287374657020DB
:1005100069646C652064656C61792C206D7365631A
:10052000290D0A24323D00202873746570207075EF
:100530006C73652C2075736563290D0A24313D00A9
:1005400024303D0024242028766965772047726294
:100550006C2073657474696E6773290D0A242320F7
:100560002876696577202320706172616D657465F6
:100570007273290D0A2447202876696577207061F7
:1005800072736572207374617465290D0A244920A1
:100590002876696577206275696C6420696E666F7C
:1005A000290D0A244E2028766965772073746172BC
:1005B00074757020626C6F636B73290D0A24783D2B
:1005C00076616C7565202873617665204772626C70
:1005D0002073657474696E67290D0A244E783D6C2A
:1005E000696E652028736176652073746172747515
:1005F0007020626C6F636B290D0A244320286368A6
:1006000065636B2067636F6465206D6F6465290D9A
:100610000A245820286B696C6C20616C61726D2013
:100620006C6F636B290D0A2448202872756E206850
:100630006F6D696E67206379636C65290D0A7E2092
:10064000286379636C65207374617274290D0A21C3
:1006500020286665656420686F6C64290D0A3F2058
:100660002863757272656E74207374617475732972
:100670000D0A6374726C2D7820287265736574207E
:100680004772626C290D0A000D0A4772626C2031B4
:100690002E3063205B27242720666F722068656CEC
:1006A000705D0D0A005D0D0A00526573746F72690A
:1006B0006E672064656661756C74730050676D20A9
:1006C000456E6400436865636B20446F6F7200443D
:1006D000697361626C656400456E61626C6564009B
:1006E00043617574696F6E3A20556E6C6F636B650C
:1006F0006400272448277C2724582720746F2075FE
:100700006E6C6F636B00526573657420746F206349
:100710006F6E74696E7565005B000D0A00486F6D41
:10072000696E67206661696C0050726F6265206651
:1007300061696C0041626F727420647572696E67E2
:10074000206379636C6500536F6674206C696D6912
:10075000740048617264206C696D697400414C4199
:10076000524D3A20000D0A00496E76616C69642092
:1007700067636F64652049443A00556E6465666935
:100780006E65642066656564207261746500556EEF
:10079000737570706F7274656420636F6D6D616ED8
:1007A00064004D6F64616C2067726F7570207669AC
:1007B0006F6C6174696F6E00436865636B20446F92
:1007C0006F72004C696E65206F766572666C6F772C
:1007D00000486F6D696E67206E6F7420656E616290
:1007E0006C656400416C61726D206C6F636B004ED0
:1007F0006F742069646C6500454550524F4D2072FE
:10080000656164206661696C2E205573696E67208E
:1008100064656661756C74730056616C7565203C27
:10082000203320757365630053657474696E6720A7
:1008300064697361626C65640056616C7565203C27
:10084000203000496E76616C696420737461746550
:100850006D656E7400426164206E756D6265722014
:10086000666F726D617400457870656374656420AD
:10087000636F6D6D616E64206C6574746572006584
:1008800072726F723A20006F6B0D0A0011241FBE46
:10089000CFEFD8E0DEBFCDBF26E0A0E0B1E001C0E1
:1008A0001D92A63DB207E1F70E9449120C94B5389B
:1008B0000C9400004398449808953B9A3C9A0C94F9
:1008C0005A049091A20591110AC0823011F4439A02
:1008D0000895813011F4449A08950C945A040895AF
:1008E000CF93DF931F92CDB7DEB79091A3059230DF
:1008F00049F089830E94B11F89810F90DF91CF91C8
:100900000C9461040F90DF91CF910895F999FECF77
:1009100092BD81BD81E08FBB80B50895F894F999AF
:10092000FECF92BD81BD81E08FBB40B54627842FAD
:10093000992787FD9095262F30E082239323892BDA
:1009400039F06F3F19F060BD84E006C084E104C057
:10095000442321F060BD84E28FBBF99A7894089516
:100960009F92AF92BF92CF92DF92EF92FF920F933E
:100970001F93CF93DF938C017A016B01C40ED51EB8
:10098000EB01912C5C01A61AB70ACE018A0D9B1DC2
:10099000CC15DD0591F0911009C0692D772767FD11
:1009A0007095272F221F2227221F01C021E0699165
:1009B000922E960E0E948E04E8CF692DC8018E0DEE
:1009C0009F1DDF91CF911F910F91FF90EF90DF90CE
:1009D000CF90BF90AF909F900C948E049F92AF9257
:1009E000BF92CF92DF92EF92FF920F931F93CF931C
:1009F000DF938B017A016C01C40ED51EEC01912CA2
:100A00005B01A81AB90AC5018C0F9D1FCC15DD0525
:100A100091F00E948604911009C0292D332727FDEB
:100A20003095232F221F2227221F01C021E0922E62
:100A3000980E8993E8CFC8018E0D9F1D0E948604F1
:100A400021E030E0981611F020E030E0C901DF919C
:100A5000CF911F910F91FF90EF90DF90CF90BF90BB
:100A6000AF909F9008958FE3EAE2F5E0DF011D92D9
:100A70008A95E9F76DE475E080E00E94072781110F
:100A800003C087E00C94C21F089566EA75E081E414
:100A900095E00C9422342F923F924F925F926F9286
:100AA0007F928F929F92AF92BF92CF92DF92EF92FE
:100AB000FF920F931F93CF93DF93CDB7DEB7AB9722
:100AC0000FB6F894DEBF0FBECDBF9F8F8E8F89E328
:100AD000E9E6F5E0DF011D928A95E9F78AE0EAE2AE
:100AE000F5E0AAE6B5E001900D928A95E1F71D8E3A
:100AF000212C312CA12CB12C19A2512C18A2662426
:100B00006394712C08E0402E9924939485E0882EFC
:100B10008D8DEE8DFF8DE80FF11D0081002309F40E
:100B200090C29FEB900F9A3110F00C946B0F8F5F77
:100B30008D8FAE01475E5F4FBE01635E7F4F8E8D2E
:100B40009F8D0E94A816882311F40C946D0FC98CF8
:100B5000DA8CEB8CFC8CC701B6010E9448380E94ED
:100B6000B035162F70E080E090E00E94DE359B01EA
:100B7000AC01C701B6010E94623420E030E048ECCD
:100B800052E40E947A370E94DD370E94B035073464
:100B900021F00D3409F450C197C1183209F432C163
:100BA000E8F4143160F4113108F0D7C0143009F4BE
:100BB0005AC008F48EC01A30D9F10C94790F1C3148
:100BC000B9F128F4163108F4F7C00C94790F1E31EE
:100BD00079F1163209F47DC00C94790F1D3309F4B4
:100BE0000BC1A8F4153309F461C040F41B3209F4B9
:100BF000ECC0113309F4E9C00C94790F1C3310F0E8
:100C00000C94790F16531093700589E000C11C35C0
:100C100040F41A3508F0B0C0103509F49BC00C94AC
:100C2000790F1C3529F01F3508F4BDC00C94790FDD
:100C30006115710531F4B8A1B1110C946F0FE1E0A9
:100C4000E8A31C3199F038F4143069F01A3009F037
:100C5000DBC082E02CC0153349F11C3559F11E313F
:100C600009F0D2C013C090926905CEC0611571051C
:100C700049F06A30710511F00C94790F24E020934B
:100C8000690509C0F3E0F093690505C061157105B8
:100C900021F48092690580E0BFC06A30710511F0CF
:100CA0000C94790F36E030936905F5CF87E0809397
:100CB0006905AAC06115710549F06A30710511F026
:100CC0000C94790F99E090936905E5CF40926905FE
:100CD000E2CFA8A1A1110C946F0FB2E0B8A312301B
:100CE00089F028F4112359F0113081F08FC01632A9
:100CF00081F0103579F1133009F088C007C01092E7
:100D00006A0584C0E8A1E0936A0580C010936A0573
:100D10007DC06E317105B1F048F46431710511F098
:100D20000C94790FF4E0F0936A0512C068327105F3
:100D300061F06233710511F00C94790F37E0309354
:100D40006A0506C080926A0503C026E020936A0502
:100D500081E062C040926A0559C0123129F0133116
:100D600039F010926E0502C090926E0582E04FC07D
:100D700082E080936E054BC06115710549F41A3508
:100D800019F410926D0502C090926D0583E044C085
:100D90006A30710511F00C94790F1A3511F40C9426
:100DA000790F84E039C01D3519F490926B0502C0AB
:100DB00010926B0585E02BC0143119F490926C05EC
:100DC00002C010926C0586E022C088A181110C94AB
:100DD0006F0F113331F410926F0588E093E098A300
:100DE0001BC06A30710511F00C94790F90926F0559
:100DF00088E0A3E0A8A310C0672B11F00C94790F32
:100E00008AE00AC087E003C080E001C081E0672B70
:100E100019F087E10C948C0FF30102C0EE0FFF1F55
:100E20008A95E2F7CF019F012A213B21232B09F468
:100E300048C085E10C948C0F672B59F7163018F4D5
:100E4000133058F017C0173010F40C94790F1A3083
:100E500000F11E3159F00C94790F123039F01E3127
:100E600029F0111125C09092710522C082E0809373
:100E700071051EC0143029F0153039F090927305B9
:100E800006C082E08093730502C0109273058CE067
:100E900010C0183029F0193039F09092720506C050
:100EA00082E08093720502C0109272058DE001C04D
:100EB0008BE0930102C0220F331F8A95E2F7C9012C
:100EC000B3CFA82AB92A24CE802F992787FD9095E1
:100ED000A92FB92FFC01E654F109E531F10510F015
:100EE0000C94790FEC5CFF4F0C949538C09274050C
:100EF000D0927505E0927605F092770580E07FC08C
:100F0000C0927805D0927905E0927A05F0927B053F
:100F100039A1316039A381E072C0C0927C05D092C2
:100F20007D05E0927E05F0927F0589A1826089A30C
:100F300082E065C0C0928005D0928105E092820572
:100F4000F092830599A1946099A383E058C010930F
:100F5000840584E054C0C701B6010E94AB3560939C
:100F6000850570938605809387059093880585E0B5
:100F700046C0C0928905D0928A05E0928B05F09216
:100F80008C0586E03CC0C0928D05D0928E05E09223
:100F90008F05F092900587E032C0C0929105D09203
:100FA0009205E0929305F092940588E028C0C092E3
:100FB0009605D0929705E0929805F0929905A52D97
:100FC000A1605A2E8AE01BC0C0929A05D0929B0560
:100FD000E0929C05F0929D05B52DB2605B2E8BE0F2
:100FE0000EC0C0929E05D0929F05E092A005F0929F
:100FF000A105E52DE4605E2E8CE001C089E083014F
:10100000082E02C0000F111F0A94E2F79801222156
:101010003321232B09F065C721E633E002C0359563
:1010200027958A95E2F720FF09C020E030E0A9016A
:10103000C701B6010E943C3587FD55C7202A312AD9
:1010400067CD552029F038A1311102C082E088A374
:1010500025FE0EC08091850590918605A09187059B
:10106000B091880580389649A849B1050CF03DC774
:1010700080916B05813031F4F8A1F230A1F520FEAA
:101080003EC731C080912B0581112DC020FE1BC0B1
:1010900080916C05813039F523E333E34BEC51E467
:1010A0006091740570917505809176059091770532
:1010B0000E947A3760937405709375058093760566
:1010C0009093770510C08091380590913905A091D3
:1010D0003A05B0913B058093740590937505A093F4
:1010E0007605B093770530FC10C08091340590915F
:1010F0003505A0913605B091370580939105909301
:101100009205A0939305B093940580916905813071
:1011100031F426FC02C08CE1FFC6E89426F88091E9
:101120006E05882341F0813061F019A682E088A71E
:1011300091E09FA30BC022E029A731E038A71FA2AE
:1011400005C0A1E0A9A718A6B2E0BFA380916C05D5
:10115000813021F0E8A1E33091F52AC0B6E9EB2E09
:10116000B5E0FB2E00E010E0C52CD12CC601002E0E
:1011700002C0959587950A94E2F780FF10C023E39B
:1011800033E34BEC51E4D7016D917D918D919C91AE
:101190000E947A37F70160837183828393830F5FA4
:1011A0001F4FF4E0EF0EF11C03301105F9F6D2CF1A
:1011B00080916F05813019F424E0521298C68CE0BA
:1011C000EDE4F5E0DE011D9601900D928A95E1F7C0
:1011D000B1FC09C0309169053E8F3230B9F038302A
:1011E00009F4B0C015C180917005873010F08DE111
:1011F00093C690913005981769F3BE01635F7F4FE6
:101200000E940727882309F484C6E4CF511002C046
:101210008AE182C6C10180759927892B09F47BCFA9
:101220006091890570918A0580918B0590918C055C
:101230000E9448380E94B0356730C8F68091840516
:10124000843129F0823009F054C627FC52C68FEA57
:101250002822662319F061506E8F03C090917005AB
:101260009E8FBE016F5F7F4F8E8D0E940727882360
:1012700009F44FC64090840560906505709066053E
:101280008090670590906805DE0111967D01F6E972
:10129000CF2EF5E0DF2EA1E4AA2EA5E0BA2E00E0C5
:1012A00010E0E52DF0E0FEA3EDA38DA19EA1002EA0
:1012B00002C0959587950A94E2F780FF33C0F4E168
:1012C0004F1226C0D50158962D913D914D915C91BC
:1012D0005B976D917D918D919C910E946234F60196
:1012E00020813181428153810E946234D7016D9304
:1012F0007D938D939C9313970230A1F4A4019301E5
:101300000E946234F70160837183828393830AC0F1
:10131000F60180819181A281B381F701808391835D
:10132000A283B3830F5F1F4FF4E0EF0EF11C24E0A4
:10133000C20ED11C34E0A30EB11C0330110509F01C
:10134000B4CF33C1552009F463CF60906505709028
:101350006605809067059090680506E915E0E1E470
:10136000CE2EE5E0DE2E5E018DE0A80EB11CE12C54
:10137000F12CA52DB0E0BF8FAE8F8E8D9F8D0E2CE2
:1013800002C0959587950A94E2F780FF26C0F50183
:101390002081318142815381D6016D917D918D9162
:1013A0009C910E946234F8012081318142815381F5
:1013B0000E946234D8016D937D938D939C93139713
:1013C000B2E0EB1214C0A40193010E946234F80150
:1013D00060837183828393830AC0F601808D918D2F
:1013E000A28DB38DF80180839183A283B383FFEF35
:1013F000EF1AFF0A0C5F1F4F24E0C20ED11C34E02D
:10140000A30EB11C83E0E816F10409F0B6CFCCC0FE
:1014100098A1933079F4AE8DA53009F48BC0A73034
:1014200009F4BDC0A33009F0BFC0BE016F5F7F4F9C
:1014300086E084C0552079F340906D058090650565
:1014400090906605A0906705B090680571E4C72E7E
:1014500075E0D72E06E915E03E01BDE06B0E711C6C
:10146000E12CF12CE52DF0E0FEA3EDA38DA19EA1D2
:101470000E2C02C0959587950A94E2F780FD0BC06B
:10148000F60180819181A281B381F80180839183EB
:10149000A283B3833EC0FE8DF730D9F1411028C03E
:1014A000D60158962D913D914D915C915B97F3013A
:1014B00060817181828193810E946334D8012D9172
:1014C0003D914D915C910E946334F801608371837A
:1014D00082839383F2E0EF121CC0A50194010E9465
:1014E0006334D8016D937D938D939C93139711C0B2
:1014F000F6012081318142815381D8016D917D9126
:101500008D919C910E946334F80160837183828382
:101510009383FFEFEF1AFF0A24E0C20ED11C0C5F89
:101520001F4F34E0630E711C83E0E816F10409F0EC
:101530009DCF71CFBE016F5F7F4F87E00E9407276D
:10154000882309F4E6C4511003C01E8E18A22DC0D2
:1015500020E030E080E090E0452D50E0BA01082E18
:1015600002C0759567950A94E2F760FD11C0F90114
:10157000E65DFA4FC788D08CE18CF28CE1E0F0E0B8
:10158000EC0FFD1FE20FF31FC082D182E282F382D3
:1015900001962C5F3F4F8330910501F705C0809184
:1015A0006A05823008F0A7C41E8E10916A051830B3
:1015B00041F4552009F4B3C198A1913009F09DC4BC
:1015C0008BC2A8A1A23009F0AAC11123D9F020E052
:1015D00030E0A901609174057091750580917605E0
:1015E000909177050E943C35882309F488C4143013
:1015F00028F4123058F4113029F06EC2183008F473
:101600004DC16AC2511068C218A28CC1552009F49C
:10161000FFCDFFA1EF2FF0E0FEA3EDA338A5232F10
:1016200030E03BA72AA781E090E03C0108A402C07B
:10163000660C771C0A94E2F70FA002C0880F991F6E
:101640000A94E2F7682A792A852D90E0862197216D
:10165000892B09F456C4CF01880F991F880F991F51
:10166000FC01E759FA4FDC01A65DBA4F57962D9160
:101670003D914D915C915A9765A576A587A590A956
:101680000E9462346B017C018AA59BA5880F991F7B
:10169000880F991FFC01E759FA4FDC01A65DBA4F8C
:1016A00057962D913D914D915C915A9765A576A5E0
:1016B00087A590A90E9462344B015C0127FE40C0BF
:1016C000E89427F820919605309197054091980568
:1016D00050919905609141057091420580914305B3
:1016E000909144050E943C35811120C120919A05BA
:1016F00030919B0540919C0550919D056091450559
:101700007091460580914705909148050E943C35AF
:1017100081110CC120919E0530919F054091A0053B
:101720005091A1056091490570914A0580914B0542
:1017300090914C050E943C358111F8C081E2ECC3C8
:10174000F9A14F2E512C64207520672809F4DBC3C2
:1017500021EF222280916C05813009F45AC00AA53C
:101760001BA5000F111F000F111F03591A4FD8019D
:101770001B962D913D914D915C911E97C501B40131
:101780000E9462342B013C01ADA0BEA0AA0CBB1C80
:10179000AA0CBB1CF501E359FA4F5F012385348580
:1017A00045855685C701B6010E946234A3019201A6
:1017B0000E9496176B017C01D8011B962D913D91DB
:1017C0004D915C911E97F50163857485858596859D
:1017D0000E9496174B015C0160938D0570938E05F6
:1017E00080938F05909390059B01AC01C701B601D2
:1017F0000E9462346B017C01E894F7F82AE037ED2F
:1018000043EA5BE3C701B6010E943F3718164CF16B
:1018100063C188E7682E85E0782E00E010E0C20101
:10182000002E02C0959587950A94E2F780FF10C0BC
:1018300023E333E34BEC51E4D3016D917D918D9122
:101840009C910E947A37F301608371838283938332
:101850000F5F1F4FF4E06F0E711C03301105F9F696
:101860007ECF20E030E040E05FE3C701B6010E9498
:101870003F3718160CF462CF2FE632E143E85AE303
:10188000C501B4010E947A379B01AC01C701B601C2
:101890000E943F3718160CF451CF1EC1552009F491
:1018A000B7CC2091960530919705409198055091BD
:1018B0009905609141057091420580914305909191
:1018C00044050E943C35811107C120919A05309151
:1018D0009B0540919C0550919D0560914505709137
:1018E000460580914705909148050E943C3581113D
:1018F000F3C020919E0530919F054091A005509125
:10190000A1056091490570914A0580914B05909120
:101910004C050E943C35882309F410CFDDC028A176
:101920002111DAC0C1018E7D9C7FD9C080916C05E8
:101930008130B1F423E333E34BEC51E460918D0546
:1019400070918E0580918F05909190050E947A3755
:1019500060938D0570938E0580938F05909390050D
:1019600040908D0550908E0560908F057090900589
:1019700020E030E040E850E4C301B2010E947A3731
:10198000A30192010E947A372B013C01A701960125
:10199000C701B6010E947A379B01AC01C301B201B5
:1019A0000E9462342B013C01A5019401C501B401E0
:1019B0000E947A379B01AC01C301B2010E946234DC
:1019C0002B013C0120E030E0A9010E943C3587FD5D
:1019D000A2C2C301B2010E9407382B013C01A5013C
:1019E0009401C701B6010E9496179B01AC01C30187
:1019F000B20190580E9443352B013C0180916A0549
:101A0000833021F477FA709477F8709480918D0583
:101A100090918E05A0918F05B091900589A39AA30E
:101A2000ABA3BCA320E030E0A901BC01CD010E9422
:101A30003C3587FF11C077FA709477F8709489A1CC
:101A40009AA1ABA1BCA1B05880938D0590938E054F
:101A5000A0938F05B09390050DA11EA1000F111F3B
:101A6000000F111F03591A4FA3019201C501B401C0
:101A70000E947A379B01AC01C701B6010E94623413
:101A800020E030E040E05FE30E947A37D8011B9607
:101A90006D937D938D939C931E970AA51BA5000FB4
:101AA000111F000F111F03591A4FA3019201C70103
:101AB000B6010E947A379B01AC01C501B4010E94B6
:101AC000633420E030E040E05FE30E947A37F801C1
:101AD0006387748785879687C1018E7D907E892B69
:101AE00009F013C28091850590918605A091870524
:101AF000B091880580933D0590933E05A0933F05E6
:101B0000B093400580916B0580932B0580917405FF
:101B100090917505A0917605B09177058093380571
:101B200090933905A0933A05B0933B05C090910579
:101B3000D0909205E0909305F0909405A70196014E
:101B40006091340570913505809136059091370587
:101B50000E943C358823C1F080913305882321F011
:101B6000B701A6010E9424298091910590919205C8
:101B7000A0919305B0919405809334059093350519
:101B8000A0933605B09337058091950580933C0569
:101B90008091730590913305981771F04091340549
:101BA0005091350560913605709137050E942429C2
:101BB0008091730580933305809172059091320571
:101BC000981731F00E94700480917205809332055D
:101BD00080916905813051F46091890570918A0581
:101BE00080918B0590918C050E94C91580916E059E
:101BF00080932E0580916C0580932C0538A133309D
:101C0000F9F480916F0580932F05813089F48091DC
:101C10009E0590919F05A091A005B091A10580938C
:101C2000650590936605A0936705B093680508C0A5
:101C3000109265051092660510926705109268056E
:101C40008091700590913005981759F08093300578
:101C50008CE0FE013D96ADE4B5E001900D928A95D1
:101C6000E1F780916D0580932D058091690590E0E5
:101C7000FC013297E830F10508F04BC0E75BFF4FFD
:101C80000C949538BE016F5F7F4F8E8D0E948F251B
:101C9000809130059E8D89133CC08CE0FE01319609
:101CA000ADE4B5E01AC0A8A1AA2349F020E040E0C5
:101CB00050E060E87FEB86E995E00E94821220E028
:101CC00040E050E060E87FEBCE0101960E94821276
:101CD0008CE0FE013196A1E4B5E001900D928A9569
:101CE000E1F717C061E475E086E003C061E475E0E8
:101CF00087E00E948F250DC08CE0E6E9F5E0A9E5BC
:101D0000B5E0EBCF8CE0E9E5F5E0DF011D928A95C7
:101D1000E9F780916A0580932A05883009F498C014
:101D2000B8A1B23009F094C090E08830910508F075
:101D300086C0FC01EF5AFF4F0C94953820E040E03C
:101D400050E060E87FEB0AC04091380550913905BA
:101D500060913A0570913B0520912B0586E995E04D
:101D60000E9482126CC0C0903805D0903905E09076
:101D70003A05F0903B0500918D0510918E0520915C
:101D80008F053091900581E08F93E9A5EF93F8A539
:101D9000FF9315C0C0903805D0903905E0903A0502
:101DA000F0903B0500918D0510918E0520918F05D7
:101DB000309190051F9289A58F9398A59F938FA02E
:101DC000A0902B0548E755E066E975E081E495E0D1
:101DD0000E94CA120F900F900F9031C040913805A9
:101DE0005091390560913A0570913B05E12C0AC08C
:101DF000409138055091390560913A0570913B0545
:101E0000EE24E39400E015C0409138055091390567
:101E100060913A0570913B05E12C0AC0409138056C
:101E20005091390560913A0570913B05EE24E39499
:101E300001E020912B0586E995E00E9400168CE0D8
:101E4000E6E9F5E0A1E4B5E001900D928A95E1F7AD
:101E50008091710580933105882309F458C00E9450
:101E6000B11F909131058091A305913041F48230EA
:101E700079F188E00E943C340E94CA1E29C091E09A
:101E800090932A0510922E0510922D0510922B0585
:101E90001092300510923305109232058230A9F06D
:101EA000BE01635F7F4F80E00E940727882389F18E
:101EB0008CE0FE013D96ADE4B5E001900D928A956F
:101EC000E1F70E947F280E945A0487E00E943D208B
:101ED000109231051CC081E01FC082E01DC088E166
:101EE0001BC089E119C084E017C08BE115C085E2F1
:101EF00013C084E111C08EE10FC08FE10DC086E1F7
:101F00000BC080E209C083E207C084E205C080E024
:101F100003C087E001C082E2AB960FB6F894DEBF43
:101F20000FBECDBFDF91CF911F910F91FF90EF902A
:101F3000DF90CF90BF90AF909F908F907F906F90E9
:101F40005F904F903F902F900895EBE6F0E08081F6
:101F5000897E8083E8E6F0E080818E7F808308952B
:101F600084B1897E84B985B1866185B98091C606C0
:101F700083FF0BC080916B00866180936B00809122
:101F8000680081608093680008950C94A50FCF923B
:101F9000DF92FF920F931F93CF93DF931F92CDB7E2
:101FA000DEB793B196718091C60686FD02C086E1C8
:101FB00098279923D9F0C12CD12CF12C01E010E005
:101FC0008C2D99830E9475289981892339F0980175
:101FD0000C2C01C0220F0A94EAF7F22A8FEFC81ADC
:101FE000D80AE3E0CE16D10459F701C0F12C8F2DA9
:101FF0000F90DF91CF911F910F91FF90DF90CF90C5
:1020000008951F920F920FB60F9211242F933F93B2
:102010004F935F936F937F938F939F93AF93BF93F0
:10202000EF93FF938091A305813049F080910001E7
:10203000811105C00E948A1683E00E944F34FF91EF
:10204000EF91BF91AF919F918F917F916F915F9130
:102050004F913F912F910F900FBE0F901F901895A9
:102060002F923F924F925F926F927F928F929F92A8
:10207000AF92BF92CF92DF92EF92FF920F931F9396
:10208000CF93DF93CDB7DEB766970FB6F894DEBF78
:102090000FBECDBF482E8091A205811158C105EA1F
:1020A00016E09E01235F3F4F1901A12CB12CC12CDA
:1020B000D12C7601642C712C8A2D0E946128D101CB
:1020C0008D931D01C3010A2C02C0959587950A9432
:1020D000E2F780FF1AC020E030E040EC5FEBF8014F
:1020E00060817181828193810E947A37688B572E3B
:1020F0004C01262F372FAC01C701B6010E943F3794
:1021000018161CF0C888D52C7401FFEFAF1ABF0A4F
:102110000C5F1F4F23E0A216B10471F68090CC062D
:102120009090CD06A090CE06B090CF0634E0388BCC
:102130005524539466EA75E0CE0101960E9422343C
:102140002090C706312CFE01319686EA95E09E8BE1
:102150008D8B80E090E000E010E0B701A6017058A0
:102160009301082E02C0359527950A94E2F720FFC7
:1021700028C00F5FAD89BE891D921D921D921C92D1
:1021800013979101082E02C0359527950A94E2F71E
:1021900020FF03C0552019F007C0552029F0C08248
:1021A000D182E282F38204C04083518362837383CD
:1021B0002DE030E02C0F3D1F280F391FD9012C9145
:1021C000122B019634962D893E892C5F3F4F3E8B12
:1021D0002D8B8330910521F6602F70E080E090E038
:1021E0000E94DC350E9407389B01AC01C501B40197
:1021F0000E947A37AB01BC011093BF05498B5A8B03
:102200006B8B7C8B0E942D1C00E020E049895A8951
:102210006B897C89CE0101960E942E190E946B2C3D
:102220000E944C295520E9F00E94C70FFE013D96FF
:1022300020E030E090E06191462F412359F0AC015D
:10224000022E02C0559547950A94E2F740FF02C05E
:10225000609516232F5F3F4F2330310561F71093B0
:10226000BF050E946B2C80910101847399F08091CD
:102270000101807329F00E948A160E94CA1E67C05D
:10228000511060C00E94C70F8421A9F784E00E940A
:10229000453404C0812F8C7109F0C4CF0E94F92B02
:1022A0000E94D7188091D0069091D1060E948B177A
:1022B00031E05326C9F020E030E040EA50E460917C
:1022C000D2067091D3068091D4069091D5060E94D3
:1022D0007A376B017C018090C8069090C906A09067
:1022E000CA06B090CB0610C0C090D206D090D306DC
:1022F000E090D406F090D5068090CC069090CD0664
:10230000A090CE06B090CF0688898150888B81112D
:1023100011CFE6EAF5E080E090E09301082E02C0DC
:10232000359527950A94E2F720FF04C010821182A8
:1023300012821382019634968330910571F70E94C0
:102340002D1C05C08091010182FFA0CF94CF66961D
:102350000FB6F894DEBF0FBECDBFDF91CF911F91B6
:102360000F91FF90EF90DF90CF90BF90AF909F9034
:102370008F907F906F905F904F903F902F90089537
:102380008F929F92AF92BF92CF92DF92EF92FF9285
:102390000F931F93CF93DF93C090C706D12C25EAEC
:1023A000E22E26E0F22E8C01C0E0D0E0C6010C2E19
:1023B00002C0959587950A94E2F7F8018080918094
:1023C000A280B38020E030E0A90180FF15C0C501E4
:1023D000B4010E943C3587FD20C0F70180819181C6
:1023E000A281B3819C01AD015058C501B4010E9486
:1023F0003F37181694F036C0C501B4010E943F372C
:1024000018165CF0F7012081318142815381C501AA
:10241000B4010E943C3587FF25C08091A305883018
:1024200099F00E948A1685E00E944F34DF91CF9187
:102430001F910F91FF90EF90DF90CF90BF90AF90E2
:102440009F908F900C94CA1E88E00E943C340E949A
:10245000CA1E8091A20581110FC08091A305811130
:10246000F6CFDFCF2196F4E0EF0EF11C0C5F1F4F8B
:10247000C330D10509F09ACFDF91CF911F910F9111
:10248000FF90EF90DF90CF90BF90AF909F908F9094
:1024900008950E94BD240E9454280E94252C0E9469
:1024A00018328EE1E2EAF5E0DF011D928A95E9F744
:1024B00081E08093A20578948091C60684FF03C0D2
:1024C00081E08093A3050E947A250E9433050E9433
:1024D00085280E945D040E94B00F0E94B81D0E94D2
:1024E000D7180E94F92B0E942D1C0E9445051092BE
:1024F000A20510920101109200011092A4050E9401
:10250000331FE1CFEF92FF920F931F93CF93DF938F
:1025100000D000D0CDB7DEB77C01122F8091C60667
:1025200085FF0BC0C70149835A836B837C830E945C
:10253000C0117C816B815A8149818091A3058230D1
:10254000F1F049835A836B837C830E94CA1E809179
:10255000A205811114C00E94261949815A816B81FC
:102560007C81882339F00E94DC1D49815A816B816E
:102570007C81E7CF00E0212FC7010E942E190F9028
:102580000F900F900F90DF91CF911F910F91FF90BF
:10259000EF9008952F923F924F925F926F927F92A9
:1025A0008F929F92AF92BF92CF92DF92EF92FF9263
:1025B0000F931F93CF93DF93CDB7DEB7E7970FB697
:1025C000F894DEBF0FBECDBF9C8B8B8B1B013A01F5
:1025D00009871A872B873C87AF8A2D961FAD2D97C9
:1025E0002E962FAD2E97298B2F963FAD2F973D8B93
:1025F00084E0889EA00111245A834983AB89BC8959
:10260000A40FB51FB98FA88F460D571D5B8F4A8F3A
:10261000FA0180809180A280B3802D913D914D91EF
:102620005C91C501B4010E9463346C8F7D8F8E8FE5
:102630009F8FF4E01F9F800111242B893C89200F7C
:10264000311F39A328A3A301400F511F5BA34AA345
:10265000DA014D905D906D907C90F901208131817F
:1026600042815381C301B2010E9463346CA37DA3F4
:102670008EA39FA3A501940150582D873E874F87B5
:10268000588BD301C201B0588D839E83AF83B88726
:10269000E981FA81E20DF31D2C8D3D8D4E8D5F8D0C
:1026A00060817181828193810E9462342B013C019F
:1026B000F101E00FF11F2CA13DA14EA15FA16081AE
:1026C0007181828193810E9462344B015C01A3017C
:1026D00092016D857E858F8598890E947A376983FE
:1026E0007A838B839C83A50194016D817E818F8188
:1026F00098850E947A379B01AC0169817A818B8130
:102700009C810E94633469837A838B839C83A501B7
:1027100094016D857E858F8598890E947A374B015B
:102720005C01A30192016D817E818F8198850E9459
:102730007A379B01AC01C501B4010E946234298142
:102740003A814B815C810E94D6342B013C019D89EA
:10275000992399F02DEB37E346E055EBC301B20125
:102760000E943F3787FD1DC02BED3FE049EC50E450
:10277000C301B2010E94623412C02DEB37E346E080
:1027800055E3C301B2010E943C35181654F02BEDFD
:102790003FE049EC50E4C301B2010E9463342B01D5
:1027A0003C018090BA069090BB06A090BC06B09009
:1027B000BD0629853A854B855C85CA01B9010E9411
:1027C0006334A50194010E9462349B01AC01C501F0
:1027D000B4010E947A370E9407384B015C0120E067
:1027E00030E040E05FE3C301B2010E947A372985FF
:1027F0003A854B855C850E947A379F77A5019401C5
:102800000E9443350E9419360E94B0357E8B6D8B35
:10281000DB01AB2B09F486C14B01A12CB12CBF8984
:10282000BB2361F0C501B4010E94DC359B01AC0102
:10283000C701B6010E947A376B017C01C501B40162
:102840000E94DC354B015C019B01AC01C301B2016C
:102850000E94433569877A878B879C87F989E4E0F2
:10286000FE9FC00111242B893C89280F391F3A8B08
:10287000298BF101E80FF91FD9012D913D914D915F
:102880005C9160817181828193810E946234A50193
:1028900094010E9443356CAB7DAB8EAB9FAB298519
:1028A0003A854B855C85CA01B9010E947A379B0144
:1028B000AC0160E070E080E090E40E9462344B0183
:1028C0005C012BEA3AEA4AE25EE369857A858B8508
:1028D0009C850E947A372B013C0120E030E040E8E3
:1028E00050E4C501B4010E9463349B01AC01C301F3
:1028F000B2010E947A3768A779A78AA79BA720E030
:1029000030E040E05FE3C501B4010E947A376CA774
:102910007DA78EA79FA7198201E010E0ED89FE89AF
:102920000E171F0709F4FEC0B981BC3008F04AC079
:102930002CA53DA54EA55FA56D817E818F819885D3
:102940000E947A374B015C0128A539A54AA55BA5F1
:102950006D857E858F8598890E947A37A5019401BF
:102960000E946334B62EA72E982E892E2CA53DA545
:102970004EA55FA56D857E858F8598890E947A37E3
:102980002B013C0128A539A54AA55BA56D817E8157
:102990008F8198850E947A379B01AC01C301B201F7
:1029A0000E9462346D877E878F87988BE981EF5F05
:1029B000E9838B2D9A2DA92DB82D8D839E83AF830E
:1029C000B8876EC0B80180E090E00E94DC352985B0
:1029D0003A854B855C850E947A374B015C010E94E9
:1029E00040356D837E838F839887C501B4010E9433
:1029F000FD374B015C01EA8DFB8D80819181A281C5
:102A0000B3819C01AD01505829833A834B835C8389
:102A1000AAA1BBA18D919D910D90BC91A02D88ABD9
:102A200099ABAAABBBAB2D813E814F8158856981A3
:102A30007A818B819C810E947A372B013C01A50110
:102A4000940168A979A98AA99BA90E947A379B0158
:102A5000AC01C301B2010E9463346D877E878F870A
:102A6000988BA501940169817A818B819C810E9458
:102A70007A374B015C012D813E814F81588568A9D1
:102A800079A98AA99BA90E947A379B01AC01C5014B
:102A9000B4010E9462346D837E838F83988719828C
:102AA0002D853E854F8558896C8D7D8D8E8D9F8DB2
:102AB0000E946334E88DF98D6083718382839383F0
:102AC0002D813E814F8158856CA17DA18EA19FA152
:102AD0000E946334A8A1B9A16D937D938D939C93BB
:102AE00013972CA93DA94EA95FA9E989FA896081AC
:102AF0007181828193810E946334A989BA896D931F
:102B00007D938D939C9313972F89B701A6018B8991
:102B10009C890E9482128091A205811121C00F5FC1
:102B20001F4FFCCE2F89B701A601C101E7960FB652
:102B3000F894DEBF0FBECDBFDF91CF911F910F91F3
:102B4000FF90EF90DF90CF90BF90AF909F908F90CD
:102B50007F906F905F904F903F902F900C948212D7
:102B6000E7960FB6F894DEBF0FBECDBFDF91CF91D1
:102B70001F910F91FF90EF90DF90CF90BF90AF909B
:102B80009F908F907F906F905F904F903F902F908D
:102B90000895CF93DF9300D000D0CDB7DEB720915A
:102BA000A305223099F069837A838B839C830E94EA
:102BB000B11F40E069817A818B819C810F900F90D9
:102BC0000F900F90DF91CF910C945A170F900F90A8
:102BD0000F900F90DF91CF9108950E94A50F84E090
:102BE0000E94301083E00E9430100E94CA1E809123
:102BF000A205811104C00E9445050C94B00F0895F0
:102C0000CF92DF92EF920F93CF93DF9300D000D05B
:102C10001F92CDB7DEB76C018091A305823009F415
:102C20006DC02D8349835A836B837C830E94B11FBF
:102C30001092BE05802F0E94A61D0E94BD1D2D81F1
:102C400049815A816B817C81882351F080E10E9407
:102C50004F340E94CA1E7C816B815A8149812D812B
:102C60008091A20581114AC0C6010E94821281E0B2
:102C70008093020182E00E943C340E94CA1E80912F
:102C8000A20581113BC08091A3058111F6CF8091EF
:102C90000201813081F4EE2051F08CE0E6EAF5E0AB
:102CA000A2EBB5E001900D928A95E1F707C080E1B3
:102CB0000E944F3403C081E08093BE051092020150
:102CC0000E94CA1E8091A205811118C00E94F92B92
:102CD0000E94D7180E942D1C66EA75E0C6010E946A
:102CE00022340F900F900F900F900F90DF91CF91A3
:102CF0000F91EF90DF90CF900C94F1210F900F90F7
:102D00000F900F900F90DF91CF910F91EF90DF9088
:102D1000CF9008958091010184FD19C080E10E9447
:102D20003C340E947F280E945A049091A305892F69
:102D30008C7021F48091A5058C7049F0943011F4C9
:102D400080E201C088E00E944F340C946829089505
:102D50006F927F928F929F92AF92BF92CF92DF92AB
:102D6000EF92FF920F931F93CF93DF937C018B0120
:102D70006A01FB018081F701E80FF11D2081EF015D
:102D80002D3229F4229621816624639407C02B32C8
:102D900011F0219602C022962181612CA12CB12C28
:102DA000712C60E070E0CB01FE0130ED932E920EAD
:102DB00029E02915C8F0B39428E02B1588F0A1105C
:102DC0007A94A5E0B0E09B01AC010E949B38660FAD
:102DD000771F881F991F690D711D811D911D0BC0E3
:102DE000A11009C0739407C02EEF921207C0A11062
:102DF00005C0AA24A39421962081D6CFBB2009F434
:102E000049C00E94DC354B015C0120E030E0A901A3
:102E10000E943C35882361F18FEF78166CF42AE02C
:102E200037ED43E25CE3C501B4010E947A374B0100
:102E30005C0173947394F0CF78120BC02DEC3CECD2
:102E40004CEC5DE3C501B4010E947A374B015C0193
:102E50000FC0772069F020E030E040E251E4C50186
:102E6000B4010E947A374B015C017A9417149CF3E9
:102E7000662021F0B7FAB094B7F8B094F6018082DA
:102E80009182A282B382CE19DF09C150F801C083BA
:102E900081E001C080E0DF91CF911F910F91FF9001
:102EA000EF90DF90CF90BF90AF909F908F907F90EA
:102EB0006F9008950F931F93CF93C42F20E030E0BD
:102EC00040EA51E40E947A370E9429350E94B035C9
:102ED0008B0101151105D9F08091A205811117C050
:102EE000C11103C00E94CA1E06C00E94DF1D80914E
:102EF000A40581FD0CC02FEF80E792E021508040B7
:102F00009040E1F700C0000001501109E2CFCF91DD
:102F10001F910F910895009741F0EFE9FFE031977D
:102F2000F1F700C000000197F6CF08958F929F92AD
:102F3000AF92BF92CF92DF92EF92FF9269017A0136
:102F40009B01AC010E947A374B015C01A7019601FD
:102F5000C701B6010E947A379B01AC01C501B401DB
:102F60000E946334FF90EF90DF90CF90BF90AF90BE
:102F70009F908F900C9407384F925F926F927F9240
:102F80008F929F92AF92BF92CF92DF92EF92FF9279
:102F90000F931F93CF93DF9310912101111101C063
:102FA00012E1115000911F01101709F4EFC089E2DE
:102FB000189FE0011124CD5DDE4F8D889E88AF887B
:102FC000B88C69A17AA18BA19CA19B01AC010E9444
:102FD00063342DA13EA14FA158A50E947A376B0101
:102FE0007C019B01AC01B401C5010E943C3587FF07
:102FF00002C064017501A601B701498B5A8B6B8B26
:103000007C8B111101C012E177247A94710E701635
:1030100019F029E2622E27C080912201081351C0C5
:103020000E94472C4EC0679C800111240D5D1E4FED
:10303000711002C092E1792E7A9480912201781267
:1030400002C00E94472CF801C588D688E788F08C1A
:10305000A701960161897289838994890E943C3510
:10306000811106C0E80180911F017812DCCF29C0D0
:10307000F80161A172A183A194A19B01AC010E94FE
:103080006334F80125A136A147A150A50E947A37E3
:1030900029893A894B895C890E9463344B015C0120
:1030A000A70196010E943C35F80187FF05C0818A7F
:1030B000928AA38AB48AD6CFC18AD28AE38AF48A52
:1030C000D1CF60901F01F9E26F9E800111240D5D48
:1030D0001E4F77247394760C82E1781201C0712C14
:1030E0005090210189E2482E751409F44DC0479C87
:1030F000E0011124CD5DDE4FF80181889288A3881C
:10310000B488C988DA88EB88FC88A7019601C501D4
:10311000B4010E943C3587FF23C0F80161A172A170
:1031200083A194A19B01AC010E946334F80125A105
:1031300036A147A150A50E947A379B01AC01C50179
:10314000B4010E9463344B015C01A70196010E9407
:103150003C3587FF05C0898A9A8AAB8ABC8A672C6E
:103160002D893E894F89588D69897A898B899C89F7
:103170000E943C35811101C0672C7394F2E17F12EB
:1031800001C0712C8E01B0CF60921F01DF91CF91F1
:103190001F910F91FF90EF90DF90CF90BF90AF9075
:1031A0009F908F907F906F905F904F9008958CE1EB
:1031B000E3E0F1E0DF011D928A95E9F71092220128
:1031C0001092210181E08093200110921F01089547
:1031D0009091220180912101891769F081E0890F86
:1031E000823109F480E020911F01921302C0809384
:1031F0001F01809322010895809122019091210165
:10320000981739F029E2829FC00111248D5D9E4FED
:10321000089580E090E00895E0912201EF5FE231AF
:1032200009F4E0E080912101E81761F089E2E89F6C
:10323000F0011124ED5DFE4F6189728983899489C3
:103240000C94073860E070E0CB01089581E0209194
:10325000220190912001291380E008952F923F923E
:103260004F925F926F927F928F929F92AF92BF9296
:10327000CF92DF92EF92FF920F931F93CF93DF9342
:10328000CDB7DEB7E9970FB6F894DEBF0FBECDBF5E
:10329000142F5FA368A779A7922E08AB2091210174
:1032A00039E2239F10011124F101ED5DFE4F1F0152
:1032B000158616861786108A15A216A217A210A6C2
:1032C000108249E956E766E97EE741A352A363A36A
:1032D00074A32CE0002319F0E6EAF5E002C0E3E075
:1032E000F1E0DE011D9601900D922A95E1F76C0147
:1032F00041E8E42E46E0F42E9E01275E3F4F3FA7B3
:103300002EA7CE010D969DA78CA75101FE013196E7
:10331000FBA7EAA700E0F60161917191819191917B
:103320006F01F70120813181428153810E947A37F8
:103330000E944A37EEA5FFA5619371938193919303
:10334000FFA7EEA7ECA5FDA541905190619071906B
:10335000FDA7ECA764197509860997092B013C01A3
:1033600097FF07C0442455243201461A570A680AB9
:10337000790AF5014182528263827482F1012585C6
:10338000368547855089421653066406750610F443
:1033900029013A01F101458656866786708A0E94A6
:1033A000DE35F70120813181428153810E9443350E
:1033B0002B013C01EAA5FBA5619371938193919345
:1033C000FBA7EAA720E030E0A9010E943C3587FF77
:1033D00008C0F1018080802F0E946B288829F101AC
:1033E0008083A3019201C301B2010E947A37F101E7
:1033F00025A136A147A150A50E946334F10165A320
:1034000076A387A390A70F5FF4E0EF0EF11C24E0F2
:10341000A20EB11C033009F07ECF0E9407386B0169
:103420007C01F10165A376A387A390A78585968586
:10343000A785B089892B8A2B8B2B09F4F2C120E058
:1034400030E0A901612F7FA188A599A50E943C3594
:1034500087FD21C0992061F0A7019601612F7FA10E
:1034600088A599A50E947A37162F7FA388A799A7C8
:1034700020E030E040E85FE3612F7FA188A599A5B7
:103480000E943C3587FF0EC010E01FA280E888A78D
:103490009FE399A707C019E9F6E7FFA326E928A744
:1034A0003EE739A7A701960160E070E080E89FE35E
:1034B0000E9443356EAB7FAB88AF99AFEFE0F1E090
:1034C000FFA7EEA72DE836E03DA72CA7CE010D966D
:1034D0009EA38DA3FE013196FBA7EAA7C12CD12C98
:1034E0007601EAA5FBA580809180A280B38020E0D0
:1034F00030E0A901C501B4010E943C35882309F4DC
:1035000081C02EA93FA948AD59ADC501B4010E94A3
:103510007A374B015C01EAA5FBA560837183828346
:1035200093839B01AC0160E070E080E89FE30E9420
:1035300043352B013C01E89477F8ECA5FDA52081EB
:10354000318142815381C301B2010E947A3769AB54
:103550007AAB8BAB9CAB9B01AC01612F7FA188A5A3
:1035600099A50E943C3587FF07C019ABFFA1FAABB4
:1035700028A52BAB39A53CABF101F1A1FFA3F101CB
:10358000F2A1F8A7F101F3A1F9A7F101F4A1FDABB4
:10359000ECA5FDA52485358546855785C301B20177
:1035A0000E947A373B018C019B01AC016FA178A589
:1035B00089A59DA90E943C3587FF04C06FA078A40F
:1035C00009A51DA9C301D801F10181A392A3A3A359
:1035D000B4A3EEA5FFA52081318142815381C501AD
:1035E000B4010E947A379B01AC01C701B6010E9469
:1035F00062346B017C0119A9FAA9FFA32BA928A7A2
:103600003CA939A78AA59BA504969BA78AA7EEA5E6
:10361000FFA53496FFA7EEA72CA53DA52C5F3F4F35
:103620003DA72CA7EDA1FEA18E179F0709F059CF4A
:103630009091210180912201981719F0F8A9FF2398
:1036400031F0F101118A128A138A148A0BC024EA1C
:1036500030E74DE75FE3C701B6010E943F37181618
:1036600034F4F101118E128E138E148E5FC024EA91
:1036700030E74DE75FEBC701B6010E943F371816F0
:1036800044F034EAC32E30E7D32E3DE7E32E3FEB80
:10369000F32EA701960160E070E080E89FE30E94AE
:1036A000623420E030E040E05FE30E947A370E941D
:1036B00007386B017C012091B6063091B706409126
:1036C000B8065091B906F10161A172A183A194A13C
:1036D0000E947A37A70196010E947A374B015C015C
:1036E000A701960160E070E080E89FE30E946234E9
:1036F0009B01AC01C501B4010E944335D62EE72ED3
:10370000F82E092F20E030E0A9010E943C3587FF08
:1037100004C0D12CE12CF12C00E04D2D5E2D6F2D3D
:10372000702FF101418F528F638F748F212F3FA132
:1037300048A559A5612F7FA188A599A50E947A3730
:10374000162F072FF82EE92E862F902FAF2DBE2D86
:10375000F101858F968FA78FB0A3A18CB28CC38CFB
:10376000D48C60901B0170901C0180901D01909082
:103770001E019301A401612F702F8F2D9E2D0E9499
:103780003C3587FD0BC09301A401B501C6010E9421
:103790003C3587FD11C0530164010EC0212F302F2D
:1037A0004F2D5E2DB501C6010E943C3587FD04C03A
:1037B000A12EB02ECF2CDE2CC501D601F101858BB8
:1037C000968BA78BB08FF8A9F1112DC08CE0FE016C
:1037D0003196AFE0B1E001900D928A95E1F7812F2B
:1037E000902FAF2DBE2D80931B0190931C01A093B1
:1037F0001D01B0931E018CE0FE017996A3E0B1E0BB
:1038000001900D928A95E1F780912001809321012A
:103810008F5F823109F480E0809320010E94BC1701
:1038200002C080E001C081E0E9960FB6F894DEBFE7
:103830000FBECDBFDF91CF911F910F91FF90EF9001
:10384000DF90CF90BF90AF909F908F907F906F90C0
:103850005F904F903F902F9008958091A605909192
:10386000A705A091A805B091A905809303019093A5
:103870000401A0930501B09306018091AA059091DF
:10388000AB05A091AC05B091AD0580930701909375
:103890000801A0930901B0930A018091AE059091AF
:1038A000AF05A091B005B091B10580930B01909345
:1038B0000C01A0930D01B0930E0108958091210198
:1038C00090912201891708F48E5E891B08950E9449
:1038D000472C8091220180931F010C94BC17CF9339
:1038E000DF93EC018991882319F00E94D324FACF49
:1038F000DF91CF910895CF93DF93FC018491EF0185
:103900002196882321F00E94D324FE01F7CFDF9176
:10391000CF910895EF92FF920F931F93CF93DF9370
:103920001F92CDB7DEB7262FEDB6FEB66DB77EB7C8
:10393000641B71090FB6F8947EBF0FBE6DBF0DB743
:103940001EB70F5F1F4F302FF8019E2F931B941748
:1039500028F4622F0E9467389193F7CF442361F0D7
:10396000F801E40FF11D31978081805D49830E9449
:10397000D32449814150F2CF0FB6F894FEBE0FBE5A
:10398000EDBE0F90DF91CF911F910F91FF90EF90BF
:10399000089548E062E00C948A1C8A3020F0843656
:1039A00020F442E003C041E001C043E06AE00C942F
:1039B0008A1C8F929F92AF92BF92CF92DF92EF922A
:1039C000FF920F931F93CF93DF93CDB7DEB72A9764
:1039D0000FB6F894DEBF0FBECDBF6B017C01142F74
:1039E00020E030E0A9010E943C3587FF07C08DE24E
:1039F0000E94D324F7FAF094F7F8F094012F0230E4
:103A000060F020E030E048EC52E4C701B6010E94CB
:103A10007A376B017C010250F2CF10FF0AC020E020
:103A200030E040E251E4C701B6010E947A376B01F1
:103A30007C0120E030E040E05FE3C701B6010E9476
:103A400063340E94AB35E1E0F0E0EC0FFD1FE10FC5
:103A5000F11D2EE22083D12C5AE0852E912CA12C31
:103A6000B12C6115710581059105A9F0D11201C034
:103A7000D394EE24E394F12CEC0EFD1EED0CF11C1E
:103A8000A50194010E947338605DF7016083B9015C
:103A9000CA01D394E6CF80E3D11648F4E1E0F0E028
:103AA000EC0FFD1FED0DF11D8083D394F5CF8D2D0F
:103AB000D1120BC0D394D3948F5FE1E0F0E0EC0F10
:103AC000FD1FE80FF11D80E38083DD2041F0FE0142
:103AD000ED0DF11D80810E94D324DA94F6CF2A9651
:103AE0000FB6F894DEBF0FBECDBFDF91CF911F910F
:103AF0000F91FF90EF90DF90CF90BF90AF909F908D
:103B00008F9008952091C60620FF08C02BE832E46C
:103B100041E25DE30E947A3744E001C043E00C9447
:103B2000D91C2091C60620FF08C02BE832E441E2F0
:103B30005DE30E947A3741E001C040E00C94D91C5B
:103B400043E00C94D91C40E00C94D91C1092C005A1
:103B50009091C60697FD03C090E29093C00588231C
:103B600031F08091C00590E289278093C0050895C7
:103B70003D98459A80E00C94A61D86B18072909184
:103B8000C00589270895809102018130A1F40E9427
:103B9000BD1D882381F0109202018CE0E6EAF5E079
:103BA000A2EBB5E001900D928A95E1F780910101B9
:103BB000806480930101089582E00C943C34CF939B
:103BC000DF93C0910001CC2339F181E08093A305FC
:103BD000C1FD0FC0C2FF02C082E00BC0C3FF02C024
:103BE00083E007C0C4FF02C084E003C0C5FF03C078
:103BF00085E00E941320C0FD04C08FEF0E9458345E
:103C00000BC081E00E943D2080E10E9445348091FC
:103C1000010184FFFCCFF1CFC0910101CC2309F455
:103C2000AEC0C4FF04C081E08093A205B0C0C0FF55
:103C300005C00E94902381E00E944534DC2FD87695
:103C400009F447C08091A305882351F0982F9C77F1
:103C5000E9F1883029F40E94472C84E08093A5057F
:103C60008091A305811106C091E09093A40592E094
:103C70009093A505C6FF0AC0883019F480E48093AC
:103C8000A3058091A40580648093A405C3FF07C0A9
:103C90008091A305803219F080E18093A305C5FFD0
:103CA00015C086E00E943D208091A405982F98724F
:103CB000983221F4837E82608093A4058091A405CC
:103CC00080628093A40580E28093A30588E60E9429
:103CD0004534C1FF38C0D11133C08091A30588237A
:103CE00031F0807569F18091A40580FF29C0809131
:103CF000A405982F9472943239F484FD02C0886030
:103D000001C08F7D8093A4058091A40585FD18C016
:103D10001092A5050E94FC18892B71F08091A405D2
:103D200086FD0AC01092A40588E08093A3050E9436
:103D30006B2C0E944C2904C01092A4051092A3057C
:103D400082E00E944534C2FF1AC08091A3058073AF
:103D500079F00E94671C9091A50592FF05C08091A3
:103D6000A40581608093A405937F9093A50504C06A
:103D70001092A4051092A30584E00E94453480911E
:103D8000A3058C7721F0DF91CF910C946B2CDF9100
:103D9000CF910895CF930E94DF1D8091A4058823C1
:103DA00009F45FC0C0E18091A405882309F459C0DB
:103DB0009091A205911155C0982F9172913209F0FE
:103DC0004DC082FD0BC00E947F280E945A04809142
:103DD000A4058D7F84608093A40540C08091A305D5
:103DE000803231F40E946F32811102C0C093A3056A
:103DF0009091A40593FF32C080913305882399F0F8
:103E000091FD11C040913405509135056091360502
:103E1000709137050E948F2841E060E070E080E8F3
:103E20009FE30E945A1780913205882369F0909190
:103E3000A40591FD09C00E94610441E060E070E0CA
:103E400080E89FE30E945A178091A40581FD06C077
:103E500080618093A40582E00E943C340E94DF1DB3
:103E6000A2CFCF910895CF93DF930E946C208091D1
:103E7000A305813021F482E00E943D2030C01092E1
:103E8000A3050E946F32882339F08091010180627E
:103E9000809301010E94CA1E85E094E00E94713265
:103EA0001EC08D3061F0CC2399F1893209F4CD7FA9
:103EB0000E9419258F3F09F448C08A3091F70E946B
:103EC000CA1E8091A205811149C0ED2FF0E0EB5F81
:103ED000FB4F1082C0FF06C08BE00E94C21FD0E0E3
:103EE000C0E0E6CF809105048823B9F3843229F439
:103EF00085E094E00E949032F0CF8091A30581305C
:103F000011F489E0EACF85E094E00E944B05E5CF0B
:103F1000813270F28F3261F2883289F08B3389F00E
:103F2000DF3488F42D2F30E0DF5F9FE9980FF9012F
:103F3000EB5FFB4F9A3108F480528083B9CFC2E027
:103F4000B7CFC4E0B5CFC1E0B3CF0E94DC1D0E9463
:103F5000CA1E8091A205882309F4AACFDF91CF91D0
:103F600008950E94DC1D0E94CA1E8091A205811145
:103F700008C00E94FC18892BB1F78091A3058830F6
:103F800091F30895CF93C82F811103C087E898E07B
:103F900047C08FE798E00E947B1C4C2F50E0FA014D
:103FA0003197E631F10598F5E75AFF4F0C949538B3
:103FB00087E698E002C085E598E00E947B1C2EC051
:103FC00083E498E0FACF89E398E0F7CF88E298E0BD
:103FD000F4CF89E198E0F1CF88EF97E0EECF8FEE54
:103FE00097E0EBCF84EE97E0E8CF81ED97E0E5CF67
:103FF00083EC97E0E2CF88EB97E0DFCF82EA97E0AF
:10400000DCCF8EE897E0D9CF8AE797E0D6CF88E675
:1040100097E00E947B1C8C2F0E94CD1C85E697E0C8
:10402000CF910C947B1CCF93C82F8DE597E00E9415
:104030007B1CC33091F03CF4C13061F0C230A1F47C
:1040400087E497E00FC0C43059F0C53069F48DE1C2
:1040500097E008C082E597E005C084E397E002C0DE
:1040600089E297E00E947B1C8AE197E00E947B1C1A
:1040700084EF91E0CF910C948B17CF93C82F88E1F8
:1040800097E00E947B1C8C2F90E0FC013197E83078
:10409000F105E8F4E159FF4F0C94953886E097E07C
:1040A00014C082EF96E011C080EE96E00EC088ED5D
:1040B00096E00BC08FEC96E008C084EC96E005C05B
:1040C0008CEB96E002C089EA96E00E947B1C85EAB0
:1040D00096E0CF910C947B1C88E896E00C947B1CB6
:1040E00084E495E00C947B1CFF920F931F93CF9375
:1040F000DF9380E495E00E947B1C8091B1060E94D2
:10410000CD1C87E295E00E947B1C8091B4060E9442
:10411000CD1C89E095E00E947B1C8091B2060E9434
:10412000CD1C80EF94E00E947B1C8091B2060E941F
:10413000C91C89EE94E00E947B1C8091B3060E940A
:10414000CD1C81ED94E00E947B1C8091B3060E94FF
:10415000C91C8AEC94E00E947B1C8091C60682FBFD
:10416000882780F90E94CD1C89EA94E00E947B1C7C
:104170008091C60686FB882780F90E94CD1C89E8BD
:1041800094E00E947B1C8091C606881F8827881FA8
:104190000E94CD1C89E694E00E947B1C8091B506AC
:1041A0000E94CD1C83E594E00E947B1C8091B506A3
:1041B0000E94C91C8BE494E00E947B1C6091B606AF
:1041C0007091B7068091B8069091B9060E94A01D23
:1041D0008BE294E00E947B1C6091BA067091BB0652
:1041E0008091BC069091BD060E94A01D80E194E0E4
:1041F0000E947B1C8091C60681700E94CD1C83EFBB
:1042000093E00E947B1C8091C60685FB882780F97D
:104210000E94CD1C88ED93E00E947B1C8091C60615
:1042200083FB882780F90E94CD1C8DEB93E00E94D0
:104230007B1C8091C606829581700E94CD1C81EA0C
:1042400093E00E947B1C8091C7060E94CD1C87E8EA
:1042500093E00E947B1C8091C7060E94C91C8FE7D7
:1042600093E00E947B1C6091C8067091C906809102
:10427000CA069091CB060E94A01D82E693E00E94A0
:104280007B1C6091CC067091CD068091CE069091FA
:10429000CF060E94A01D85E493E00E947B1C8091C4
:1042A000D0060E94CD1C86E293E00E947B1C6091A8
:1042B000D2067091D3068091D4069091D5060E94C3
:1042C000A01D89E093E00E947B1C6091BE06709166
:1042D000BF068091C0069091C1060E94A31D88EF81
:1042E00092E00E947B1C6091C2067091C30680918F
:1042F000C4069091C5060E94A31D8BEE92E00E9419
:104300007B1C84E6F82E10E0C1E8D6E000E089EEE0
:1043100092E00E947B1C802F8F0D0E94CD1C87EEA7
:1043200092E00E947B1C123071F01330B9F0113012
:1043300029F0688179818A819B8117C06C857D8590
:104340008E859F8512C020E030E041E655E4688DFF
:10435000798D8A8D9B8D0E94433507C08CA19DA1CC
:10436000AEA1BFA1BC01CD0190580E94A01D84EE5A
:1043700092E00E947B1C013029F0023031F082EE85
:1043800092E005C080EE92E002C08EED92E00E94C5
:104390007B1C123051F0133059F0113019F084EDBC
:1043A00092E008C082EC92E005C081EB92E002C08E
:1043B00081EA92E00E947B1C8DE992E00E947B1CC6
:1043C0000F5F2496033009F0A2CF8AE0F80E1F5F3A
:1043D0008CE8F81299CFDF91CF911F910F91FF9048
:1043E0000895CF9387E992E00E947B1CC0E06C2F78
:1043F00082EB95E00E9408340E94821DC23021F0B9
:1044000085E992E00E947B1CCF5FC33081F783E98E
:1044100092E00E947B1C8091BE050E94CD1C8FE81B
:1044200092E0CF910C947B1CEF92FF920F931F931D
:10443000CF93DF93CDB7DEB72C970FB6F894DEBFDE
:104440000FBECDBFF12CBE016F5F7F4F8F2D0E943D
:104450000727811104C087E00E94C21F69C08CE851
:1044600092E00E947B1C86E0F81631F0E7E0FE1235
:1044700008C086E892E002C089E892E00E947B1CB6
:1044800004C086E38F0D0E94CD1C84E892E00E9458
:104490007B1C8E010F5F1F4FE12CF8016191719120
:1044A000819191918F010E94821DF2E0EF1619F027
:1044B00082E892E002C08EE792E00E947B1CE394C7
:1044C00083E0E812EACFF394E8E0FE12BCCF88E77D
:1044D00092E00E947B1C09E515E0F12CF801619146
:1044E0007191819191918F010E94821DF2E0FF16DE
:1044F00019F086E792E002C082E792E00E947B1CFE
:10450000F39483E0F812EACF8CE692E00E947B1CE1
:1045100060916505709166058091670590916805C9
:104520000E94821D88E692E00E947B1C0E94F1217D
:104530002C960FB6F894DEBF0FBECDBFDF91CF91A2
:104540001F910F91FF90EF90089586E692E00E94F0
:104550007B1C80912A05823091F038F4882361F029
:104560008130A9F480E692E00CC0833069F0883095
:1045700071F486E592E005C083E692E002C08DE525
:1045800092E00E947B1C0CC08AE592E0FACF81E5A4
:1045900092E00E947B1C80912A0582500E94CD1CD3
:1045A0008EE492E00E947B1C809130058A5C0E9420
:1045B000CD1C80912E05813049F028F0823051F4D5
:1045C0008FE392E005C089E492E002C084E492E0C7
:1045D0000E947B1C80912C05811103C08AE392E02C
:1045E00002C085E392E00E947B1C80912D05811121
:1045F00003C080E392E002C08BE292E00E947B1C49
:1046000080912B05813019F486E292E002C081E2AC
:1046100092E00E947B1C80913105813049F028F0A6
:10462000823051F485E192E005C08DE192E002C054
:1046300089E192E00E947B1C80913305813031F04A
:1046400040F0823051F48DE092E005C081E192E0CB
:1046500002C089E092E00E947B1C8091320581308B
:1046600049F028F0823051F481E092E005C085E005
:1046700092E002C08DEF91E00E947B1C8AEF91E0F6
:104680000E947B1C80913C050E94CD1C87EF91E02D
:104690000E947B1C609138057091390580913A0524
:1046A00090913B050E94911D84EF91E00E947B1C3C
:1046B00060913405709135058091360590913705EC
:1046C0000E94A31D80EF91E00C947B1C1F93CF935D
:1046D000DF93182FEB018DEE91E00E947B1C812F60
:1046E0000E94CD1C8BEE91E00E947B1CCE010E94AB
:1046F0006F1C88EE91E0DF91CF911F910C947B1C91
:10470000CF93DF93EC0188ED91E00E947B1CCE01FA
:104710000E946F1C84ED91E0DF91CF910C947B1C83
:10472000BF92CF92DF92EF92FF920F931F93CF939E
:10473000DF93CDB7DEB768970FB6F894DEBF0FBE34
:10474000CDBF8CE0E6EAF5E0DE011D9601900D920A
:104750008A95E1F78091A3058430E9F040F4813037
:10476000E9F080F0823009F58FEA91E01CC08031D9
:1047700079F018F4883049F018C0803291F0803414
:1047800021F013C08EEC91E00EC089EC91E00BC0DB
:1047900083EC91E008C08DEB91E005C086EB91E0E1
:1047A00002C089EA91E00E947B1C8091B50683706B
:1047B00039F0BE01635F7F4FCE0101960E94223423
:1047C0008091B50680FD05C08091B50681FF6DC062
:1047D0001FC082EA91E00E947B1C69817A818B81F3
:1047E0009C810E94821D80EA91E00E947B1C6D8169
:1047F0007E818F8198850E94821D80EA91E00E94CF
:104800007B1C69857A858B859C850E94821DDCCF07
:1048100089E991E00E947B1C9DE4E92E95E0F92E48
:104820008E010F5F1F4FB12C6801F70161917191EB
:10483000819191917F0120853185428553850E9428
:1048400063349B01AC01F8016081718182819381A5
:104850000E946234F8016083718382839383F2E063
:10486000BF120FC020916505309166054091670524
:10487000509168050E946234F801608371838283DD
:1048800093830C5F1F4FF601608171818281938158
:104890000E94821DF2E0BF1621F087E991E00E949C
:1048A0007B1CB39423E0B212BFCF8091B50682FF88
:1048B00008C081E991E00E947B1C0E945E1C0E945E
:1048C000CD1C8091B50683FF08C08CE891E00E9462
:1048D0007B1C0E94B4240E94CD1C8091B506807779
:1048E00079F186E891E00E947B1C8091B50684FFF7
:1048F00006C00E94C70F43E062E00E948A1C84E861
:1049000091E00E947B1C8091B50685FF0BC00E9440
:10491000BD1D882319F082E891E002C080E891E093
:104920000E947B1C8EE791E00E947B1C8091B50663
:1049300086FF06C00E94293243E062E00E948A1C82
:104940008AE791E00E947B1C68960FB6F894DEBF60
:104950000FBECDBFDF91CF911F910F91FF90EF90D0
:10496000DF90CF90BF9008959091570480915804A4
:10497000891708F48058891B0895E0ECF0E08081E5
:10498000826080831092C50080E18093C400E1ECD6
:10499000F0E0808180618083808188608083808175
:1049A000806880830895E091560491E09E0F9034D2
:1049B00009F490E020915504921305C02091010163
:1049C00024FFF8CF0895F0E0EF53FA4F80839093DF
:1049D00056048091C10080628093C10008951F92A7
:1049E0000F920FB60F9211248F939F93EF93FF9323
:1049F00080915504E82FF0E0EF53FA4F90819093A7
:104A0000C6008F5F803409F480E080935504909154
:104A10005604891305C08091C1008F7D8093C10029
:104A2000FF91EF919F918F910F900FBE0F901F906C
:104A300018959091570480915804891761F0E92FD7
:104A4000F0E0EF5FF94F80819F5F903809F490E0CC
:104A50009093570408958FEF08951F920F920FB609
:104A60000F9211242F933F934F935F936F937F93F4
:104A70008F939F93AF93BF93EF93FF938091C60063
:104A80008F3369F030F4883181F0813289F488E025
:104A900009C0803431F08E3759F482E003C081E0E0
:104AA00001C080E20E943C3414C00E948A1611C0EA
:104AB000E091580491E09E0F903809F490E0209125
:104AC0005704921731F0F0E0EF5FF94F8083909335
:104AD0005804FF91EF91BF91AF919F918F917F917A
:104AE0006F915F914F913F912F910F900FBE0F905B
:104AF0001F9018958091580480935704089521E5DC
:104B0000829FC001112440E550E09D5F0C94B004E9
:104B100040E550E0BC018EEA93E00C94B0042DE037
:104B2000829FC00111244CE050E09E5F0C94B004C1
:104B30006AE080E090E00E948E0445E550E061E884
:104B400076E081E090E00C94B004EF92FF920F9336
:104B50001F93CF93DF93CDB7DEB72C970FB6F894A2
:104B6000DEBF0FBECDBF182F80FFEDC08AE080935F
:104B7000B1068FEF8093B4061092B20623E0209323
:104B8000B3062093B5068AE097EDA3EABCE38093D1
:104B9000B6069093B706A093B806B093B9068FE611
:104BA00092E1A3E0BBE38093BA069093BB06A09387
:104BB000BC06B093BD0680E090E8ABE3B6E480931A
:104BC000BE069093BF06A093C006B093C106109294
:104BD000C2061092C3061092C4061092C506209316
:104BE000C70680E090E0A8ECB1E48093C8069093FB
:104BF000C906A093CA06B093CB0680E090E8ABE369
:104C0000B4E48093CC069093CD06A093CE06B093E7
:104C1000CF068AEF90E09093D1068093D00680E093
:104C200090E0A0E8BFE38093D2069093D306A093D0
:104C3000D406B093D5061092C60640E050E060E27C
:104C400072E44093810650938206609383067093CA
:104C5000840640938506509386066093870670937A
:104C6000880685E592EFACE3B3E4809389069093E0
:104C70008A06A0938B06B0938C0640E050E06AEF62
:104C800075E440938D0650938E0660938F06709363
:104C9000900640939106509392066093930670930A
:104CA000940680E090E0AAEFB3E480939506909399
:104CB0009606A0939706B093980640E05AEB6BEDEA
:104CC00079E44093990650939A0660939B067093FB
:104CD0009C0640939D0650939E0660939F0670939A
:104CE000A00680E098ECAFE2B8E48093A106909330
:104CF000A206A093A306B093A40680E090E0A9E3E7
:104D0000B4EC8093A5069093A606A093A706B09353
:104D1000A80680E090E8A5E4B4EC8093A9069093FF
:104D2000AA06A093AB06B093AC0680E090E0A8EC96
:104D3000B2EC8093AD069093AE06A093AF06B0930D
:104D4000B0060E94982511FF10C0CE0101967C018B
:104D50008CE0F70111928A95E9F700E0B701802F06
:104D60000E948F250F5F0830C9F712FF0AC060E06C
:104D700080E093E00E948E0460E081E593E00E9471
:104D80008E0413FF05C060E08EEA93E00E948E045B
:104D90002C960FB6F894DEBF0FBECDBFDF91CF913A
:104DA0001F910F91FF90EF9008951F93CF93DF9382
:104DB000182FEB0181E5189FB00111247D5F40E5BC
:104DC00050E0CE010E94EE04892B39F41882BE0116
:104DD000812F0E947F2580E001C081E0DF91CF918B
:104DE0001F910895CF93DF93EC0140E550E06EEA08
:104DF00073E00E94EE04892B31F41882CE010E94E8
:104E0000882580E001C081E0DF91CF9108951F9354
:104E1000CF93DF93182FEB018DE0189FB001112481
:104E20007E5F4CE050E0CE010E94EE04892B59F4E5
:104E30008CE0FE0111928A95E9F7BE01812F0E9454
:104E40008F2580E001C081E0DF91CF911F9108950F
:104E500080E090E00E9486048A3059F445E550E0F5
:104E600061E070E081E896E00E94EE0421E0892B89
:104E700009F420E0822F0895CF92DF92EF92FF9203
:104E8000CF93DF93C82F6A017B0120E030E0A901B6
:104E9000C701B6010E943C3587FDF8C0C43608F44E
:104EA00045C02CE92C0F80E02330B8F530E082308B
:104EB00079F0F901EE0FFF1FEE0FFF1F833011F1A4
:104EC000813019F0EF57F94F23C0E357F94F20C055
:104ED000E901CC0FDD1FCC0FDD1FC756D94F20E0F5
:104EE00030E040E752E4C701B6010E947A3720E083
:104EF00030E040E752E40E947A37688379838A83FE
:104F00009B83C0C0EB55F94FF7FAF094F7F8F09493
:104F1000C082D182E282F382B5C08F5F2A3008F46A
:104F2000B7C0843009F4B4C02A50BECFC701B6015F
:104F30000E9448380E94B0358C2F90E08032910555
:104F400008F0A6C0FC01E958FF4F0C949538633077
:104F500008F4A0C06093B10695C06093B40692C0F7
:104F60006093B20602C06093B3060E94BD2B8AC054
:104F70008091C606662311F0846007C08B7F05C050
:104F80008091C606662321F080648093C6067AC0AD
:104F90008F7BFBCF8091C606662311F08068F5CF2A
:104FA0008F77F3CF6093B5066DC0C092B606D092EE
:104FB000B706E092B806F092B90664C0C092BA068D
:104FC000D092BB06E092BC06F092BD065BC0809119
:104FD000C606662311F08160D8CF8E7FD6CF809130
:104FE000C606662321F084FF57C08062CECF8F7D36
:104FF000CCCF8091C606662311F0886001C0877F00
:105000008093C6060E94B00F3DC08091C6066623FD
:1050100011F08061BACF8F7CB8CF6093C70632C0E1
:10502000C092C806D092C906E092CA06F092CB069A
:1050300029C0C092CC06D092CD06E092CE06F09266
:10504000CF0620C070E07093D1066093D0061AC0DE
:10505000C092D206D092D306E092D406F092D50642
:1050600011C0C092BE06D092BF06E092C006F09278
:10507000C10608C0C092C206D092C306E092C40620
:10508000F092C5060E94982580E007C084E005C024
:1050900083E003C086E001C08AE0DF91CF91FF90FA
:1050A000EF90DF90CF9008950E942827811108C0CB
:1050B00087E00E94C21F8FEF0E94A5250C947420E8
:1050C0000895882321F0813021F488E0089584E058
:1050D000089580E10895882321F0813021F480E44F
:1050E000089580E2089580E80895882321F08130B2
:1050F00021F484E0089582E0089580E10895E0EBD2
:10510000F0E080818F7780830895239A83E08093F5
:10511000B00082E08093B100259A0C947F288F9292
:105120009F92AF92BF92CF92DF92EF92FF920F9336
:105130001F93CF93DF936A017B019091A205911198
:1051400076C081110EC0DF91CF911F910F91FF901A
:10515000EF90DF90CF90BF90AF909F908F900C9486
:105160007F28813011F42D9801C02D9AA090BE06A1
:10517000B090BF060091C0061091C1068090C20693
:105180009090C306D091C406C091C50694014D2FDE
:105190005C2FB501C8010E943C3518160CF03FC0C9
:1051A0009501A801B601C7010E943F37181614F4F3
:1051B0006501780194014D2F5C2FB601C7010E9453
:1051C0003C3587FF03C06401ED2EFC2E94014D2F6A
:1051D0005C2FB601C7010E9462346B017C0194010F
:1051E0004D2F5C2FB501C8010E9462349B01AC01B8
:1051F00060E070E08FE793E40E9443359B01AC01CF
:10520000C701B6010E947A3720E030E040E05FE35A
:105210000E9463340E9419360E94B03501C06FEFBE
:105220006093B3008091B00080688093B000DF91FC
:10523000CF911F910F91FF90EF90DF90CF90BF9093
:10524000AF909F908F900895CF93DF9300D000D0C0
:105250001F92CDB7DEB79091A3059230A9F04A8393
:105260005B836C837D8389830E94B11F4A815B814C
:105270006C817D8189810F900F900F900F900F901E
:10528000DF91CF910C948F280F900F900F900F907B
:105290000F90DF91CF9108958091C60682FF02C0E2
:1052A000289A01C028988091890480939D04809158
:1052B0008A0480939C048091B106880F8450819564
:1052C00080939B0480916F00826080936F000895AB
:1052D00080916F008D7F80936F0080918100887F27
:1052E000816080938100109288048091B4068F3F82
:1052F00021F490910001992349F09091A3059430F5
:1053000029F090E00E948B1781E001C080E090912D
:10531000C60692FF02C091E08927882311F0289ADF
:105320000895289808951F920F920FB60F92112496
:105330002F933F934F935F936F937F938F939F939D
:10534000AF93BF93CF93DF93EF93FF938091880444
:105350008111EAC19BB180919D04807E9F71892B50
:105360008BB98BB1837E90919C04892B8BB98091F2
:105370009B0486BD82E085BD81E08093880478949B
:105380008091AF049091B004892B09F09FC0809167
:105390008D0490918C04981709F492C0E0918D04CB
:1053A00086E0E89FF0011124EF54FB4FF093B00426
:1053B000E093AF0483819481909389008093880067
:1053C000808191819093AB048093AA04A281809103
:1053D000AC048A1771F1A093AC0481E1A89FD001BD
:1053E0001124AB52BB4FB093AE04A093AD041D96F5
:1053F0008D919D910D90BC91A02DB695A7959795F7
:1054000087958093960490939704A0939804B09303
:1054100099048093920490939304A0939404B0937E
:10542000950480938E0490938F04A0939004B0937E
:105430009104C091AD04D091AE048091890498810B
:10544000892780939D04258189819A81AB81BC81C4
:10545000022E04C0B695A795979587950A94D2F722
:1054600080939E0490939F04A093A004B093A10402
:105470008D819E81AF81B885022E04C0B695A79517
:10548000979587950A94D2F78093A2049093A304EA
:10549000A093A404B093A50489859A85AB85BC85A7
:1054A00004C0B695A795979587952A95D2F78093CE
:1054B000A6049093A704A093A804B093A90406C0DF
:1054C0000E94682984E00E943C342EC10E94C31DC2
:1054D00010929C0480919E0490919F04A091A0043E
:1054E000B091A10440918E0450918F04609190047A
:1054F00070919104840F951FA61FB71F80938E048F
:1055000090938F04A0939004B0939104E091AD0424
:10551000F091AE044585568567857089481759070F
:105520006A077B0768F524E020939C04458556852F
:1055300067857089841B950BA60BB70B80938E042F
:1055400090938F04A0939004B09391042081809154
:10555000A6059091A705A091A805B091A90525FFE2
:1055600004C00197A109B10903C00196A11DB11D95
:105570008093A6059093A705A093A805B093A905CD
:105580008091A2049091A304A091A404B091A504D9
:105590004091920450919304609194047091950409
:1055A000840F951FA61FB71F8093920490939304B6
:1055B000A0939404B09395044585568567857089BA
:1055C000481759076A077B0778F520919C042860E3
:1055D00020939C044585568567857089841B950BAF
:1055E000A60BB70B8093920490939304A09394041A
:1055F000B093950420818091AA059091AB05A0916C
:10560000AC05B091AD0526FF04C00197A109B10911
:1056100003C00196A11DB11D8093AA059093AB050F
:10562000A093AC05B093AD058091A6049091A7041A
:10563000A091A804B091A9044091960450919704B8
:105640006091980470919904840F951FA61FB71F4D
:105650008093960490939704A0939804B093990430
:105660004585568567857089481759076A077B07FE
:1056700078F520919C04206120939C0445855685F3
:1056800067857089841B950BA60BB70B80939604D6
:1056900090939704A0939804B093990420818091EB
:1056A000AE059091AF05A091B005B091B10527FF6F
:1056B00004C00197A109B10903C00196A11DB11D44
:1056C0008093AE059093AF05A093B005B093B1055C
:1056D0008091A305843039F48091BF0590919C049A
:1056E000892380939C048091AA049091AB04019734
:1056F0009093AB048093AA04892B69F41092B004B0
:105700001092AF0480918D048F5F80938D0486305A
:1057100011F410928D0480918A0490919C04892741
:1057200080939C0410928804FF91EF91DF91CF91B8
:10573000BF91AF919F918F917F916F915F914F91A9
:105740003F912F910F900FBE0F901F9018951F92B1
:105750000F920FB60F9211248F939F939BB180915C
:105760008A048C71937E892B8BB915BC9F918F9184
:105770000F900FBE0F901F901895FF920F931F93DD
:10578000CF93DF9310928A0410928904C0E0D0E096
:105790000C2F1C2F2091B20630E08C2F0C2E02C053
:1057A000359527950A94E2F720FF07C0F0908A0408
:1057B0000E9461288F2980938A042091B30630E0EB
:1057C00002C0359527951A95E2F720FF08C0109181
:1057D0008904802F0E946B28812B80938904219655
:1057E000C330D105A9F6DF91CF911F910F91FF90A2
:1057F00008950E9468298BE2E9E5F4E0DF011D923B
:105800008A95E9F783E2EEE8F4E0DF011D928A95DC
:10581000E9F7109287041092860410928D0410927A
:105820008C0481E080938B04109288040E94BD2B2D
:105830008BB1837E90918A04892B8BB98BB18F7148
:1058400090918904892B8BB908958AB18C618AB9AA
:10585000209A8AB1806E8AB9E1E8F0E080818F7E7B
:105860008083808188608083E0E8F0E080818C7FA5
:10587000808380818F708083EEE6F0E08081887F76
:10588000808314BC15BC8081816080830895CF9390
:10589000DF93C0918604D09187042097C9F080914E
:1058A0005A04816080935A0460917004709171046D
:1058B00080917204909173049B01AC010E947A372D
:1058C000698B7A8B8B8B9C8B109287041092860449
:1058D000DF91CF9108952F923F924F925F926F92F6
:1058E0007F928F929F92AF92BF92CF92DF92EF9270
:1058F000FF920F931F93CF93DF93CDB7DEB7E5975A
:105900000FB6F894DEBF0FBECDBF8091A50581FD17
:1059100076C590918D0480918B04981709F46FC51A
:105920008091860490918704892B09F042C20E94DD
:10593000FC181C019093870480938604009709F457
:105940005EC580915A041091A50580FF03C0109296
:105950005A04B9C0E0915904EF5FE53009F4E0E082
:10596000E093590421E12E9FF0011124EB52FB4FEB
:10597000F0938504E0938404D1018C918083119687
:105980004D915D916D917C91149703E0440F551FEB
:10599000661F771F0A95D1F741835283638374830F
:1059A00015964D915D916D917C91189783E0440F10
:1059B000551F661F771F8A95D1F7458356836783E6
:1059C000708719964D915D916D917C911C9793E034
:1059D000440F551F661F771F9A95D1F7418752874D
:1059E000638774871D966D917D918D919C915097E1
:1059F0006B017C0123E0CC0CDD1CEE1CFF1C2A9506
:105A0000D1F7C586D686E786F08A0E94DC3560939A
:105A10005F04709360048093610490936204F101C9
:105A200025A136A147A150A50E9443359B01AC0199
:105A30006093630470936404809365049093660498
:105A400060E070E080EA9FE30E9443356093670462
:105A5000709368048093690490936A0410925B04C5
:105A600010925C0410925D0410925E0412FF1CC040
:105A7000609178047091790480917A0490917B040C
:105A80006093700470937104809372049093730414
:105A90009B01AC010E947A37D10151966D937D93A1
:105AA0008D939C9354970FC0F1016189728983890A
:105AB00094890E94073860937004709371048093F6
:105AC00072049093730410926C0410926D041092FF
:105AD0006E0410926F04D10191968D909D90AD90BF
:105AE000BC909497A501940160E070E080E09FE392
:105AF0000E9443352B013C01F101C5A0D6A0E7A0CF
:105B0000F0A412FF4DC0F2E0F0936B04D101519666
:105B10002D913D914D915C91549729833A834B830C
:105B20005C830E947A379B01AC01C701B6010E94D9
:105B300062342B013C0120E030E0A9010E943C3599
:105B400087FF1DC0A5019401C501B4010E94633403
:105B5000A70196010E947A379B01AC0169817A8185
:105B60008B819C810E9462340E9407386093780484
:105B70007093790480937A0490937B041AC14092C5
:105B80006C0450926D0460926E0470926F041092D7
:105B900078041092790410927A0410927B0409C15F
:105BA00010926B04C0927C04D0927D04E0927E043B
:105BB000F0927F040E940C194B015C016093780401
:105BC0007093790480937A0490937B049B01AC01D9
:105BD0000E947A376D837E838F8398870091860435
:105BE00010918704D80195962D913D914D915C912E
:105BF000989729873A874B875C8751962D913D91DD
:105C00004D915C91549729833A834B835C839B012C
:105C1000AC0169817A818B819C810E9462349B01F5
:105C2000AC01C301B2010E947A379B01AC016985C6
:105C30007A858B859C850E94633420E030E040E0CB
:105C40005FE30E947A376B017C0120E030E0A9011C
:105C50000E943F3718160CF09CC029853A854B8569
:105C60005C85C701B6010E943C3587FF8EC0F801F4
:105C7000858C968CA78CB0A02D813E814F81588554
:105C8000C501B4010E9462349B01AC01C301B201A1
:105C90000E947A3760938004709381048093820419
:105CA00090938304A70196010E943C3587FF3DC075
:105CB000C501B4010E9407386093740470937504A1
:105CC0008093760490937704A501940169817A8189
:105CD0008B819C810E943C35811104C0F1E0F093DE
:105CE0006B0467C029813A814B815C81C501B40195
:105CF0000E9462349B01AC01C301B2010E947A3759
:105D00009B01AC0160917C0470917D0480917E04C4
:105D100090917F040E94623460937C0470937D04B0
:105D200080937E0490937F0444C0C0927C04D09200
:105D30007D04E0927E04F0927F04C0928004D092B1
:105D40008104E0928204F0928304D80191966D91CF
:105D50007D918D919C9194979B01AC010E9463343D
:105D6000A70196010E947A372D813E814F81588587
:105D70000E9463340E940738609374047093750422
:105D8000809376049093770414C0B2E0B0936B04D0
:105D900010C010927C0410927D0410927E04109228
:105DA0007F048092740490927504A0927604B0925D
:105DB000770480918C04F6E0F89FF0011124EF54F1
:105DC000FB4FFA87E98780915904828320918604EA
:105DD000309187043F872E87D9019596BC91BCA747
:105DE000F901F6A1FDA7D9019796BC91BEA7F901CB
:105DF000F0A5FFA7209167043091680440916904E1
:105E000050916A046CA57DA58B2F9F2F0E94623450
:105E100068A779A78AA79BA720E030E0A9010E9484
:105E20003C3587FF04C018A619A61AA61BA6209108
:105E30007C04288F30917D04398F40917E044A8FF5
:105E400050917F045B8F809174048C8F90917504C6
:105E50009D8FA0917604AE8FB0917704BF8FE091B3
:105E60008004E8A3F0918104F9A3209182042AA37D
:105E7000309183043BA340916C044CA350916D047A
:105E80005DA380916E048EA390916F049FA3A09157
:105E90007804A8ABB0917904B9ABE0917A04EAAB8D
:105EA000F0917B04FBAB2091700429833091710445
:105EB0003D83209072043090730440916B044D87B1
:105EC0005CA5588B8DA5898B9EA59A8BAFA5AB8BB6
:105ED0003EE3C32E33ECD32E3EE2E32E39E3F32E22
:105EE000412C512C3201CC8ADD8AEE8AFF8A3D8515
:105EF000332321F0313009F47CC0B1C0AE85BF85B9
:105F000091962D913D914D915C919497C701B60169
:105F10000E947A374B015C0120E030E040E05FE313
:105F20000E947A379B01AC0169817D81C1010E9489
:105F300063349B01AC01C701B6010E947A379B0113
:105F4000AC01688979898A899B890E9462348B01B6
:105F50008DAB9CAB288D398D4A8D5B8D0E943C3575
:105F600087FF3FC0288D398D4A8D5B8D6CA57DA53F
:105F70008EA59FA50E9462349B01AC010E946334F0
:105F80006B017C012C8D3D8D4E8D5F8D69817D81F6
:105F9000C1010E9463349B01AC01C701B6010E949C
:105FA00043356B017C0128A139A14AA15BA1688D11
:105FB000798D8A8D9B8D0E943C35882319F0B1E044
:105FC000BD8702C0E2E0ED87FC8DF9832D8D2D8326
:105FD0002E8C3F8C088D198D3A8D3DAB4B8D4CAB83
:105FE000B5C0A501940169817D81C1010E9463341E
:105FF0007CC0A70196016C8D7D8D8E8D9F8D0E943A
:106000007A379B01AC01688979898A899B890E94CA
:1060100062348B018DAB9CAB28A139A14AA15BA155
:106020000E943C3587FF92C028A139A14AA15BA1FB
:10603000688979898A899B890E9462342C8D3D8D7B
:106040004E8D5F8D0E9443356B017C0108A119A123
:106050005AA15DAB8BA18CAB92E09D8777C0AE85DA
:10606000BF8591962D913D914D915C919497C7017B
:10607000B6010E947A374B015C019B01AC0169813A
:106080007D81C1010E943F3718169CF520E030E069
:1060900040E05FE3C501B4010E947A379B01AC0187
:1060A00069817D81C1010E9462349B01AC01C701FD
:1060B000B6010E947A379B01AC01688979898A8987
:1060C0009B890E9462348B018DAB9CAB2CA13DA1BE
:1060D0004EA15FA10E943F3718165CF4A501940100
:1060E00069817D81C1010E94623469837D831C01C5
:1060F0002DC02CA13DA14EA15FA1688979898A8913
:106100009B890E9462349B01AC010E9463346B0145
:106110007C0128A939A94AA95BA969817D81C101AE
:106120000E9463349B01AC01C701B6010E94433554
:106130006B017C01B8A9B983E9A9ED832AA83BA822
:106140000CA11DA1FEA1FDAB2FA12CABA7019601B7
:10615000C301B2010E9463342B013C012C893D89AB
:106160004E895F890E943C3587FF07C0A3019201D9
:106170006C897D898E899F895EC028A539A54AA52D
:106180005BA5B8018DA99CA90E943F3718160CF495
:1061900042C089819D81D1018093700490937104E4
:1061A000A0937204B09373043D8530936B042091E7
:1061B0006304309164044091650450916604B80111
:1061C0008DA99CA90E947A3769837A838B839C83EB
:1061D0000E9429356B017C0160915F04709160041D
:1061E00080916104909162040E9429354B015C0109
:1061F000A70196010E9462340E94B0356D837E83B0
:106200008F839887ED81FE81A985BA85ED93FC93F4
:10621000309741F12BC02EE333EC4EE259E36C8909
:106220007D898E899F890E9463346C8B7D8B8E8BD8
:106230009F8BA30192010E9462346B017C012CA10F
:106240003DA14EA15FA1B8018DA99CA90E943F3735
:1062500018160CF09ECF088B198B4DA94A8B5CA9A0
:106260005B8B45CE8091A50582FDBEC020915B046D
:1062700030915C0440915D0450915E04C301B20111
:106280000E9463342B013C0129813A814B815C815E
:10629000C501B4010E9462349B01AC01C301B2018B
:1062A0000E9443354B015C0120EC31EE44E65EE494
:1062B0000E947A370E9429350E94B035603DA7E0E0
:1062C0007A078105910520F4E985FA85158231C0A8
:1062D000603AFFE07F078105910510F4E1E009C015
:1062E0006034FFE17F078105910510F4E2E001C011
:1062F000E3E0A985BA851596EC93A985BA8515962C
:106300002C911597022E04C09695879577956795E1
:106310000A94D2F7ED81FE8102C0EE0FFF1F2A958D
:10632000E2F7ED93FC9361157105F1E08F0791059C
:1063300038F4A985BA8514967C936E93139706C09A
:106340002FEF3FEFE985FA853483238380918B0417
:1063500080938C048F5F863019F080938B0402C089
:1063600010928B04E0918604F0918704C801ADA9D6
:10637000BCA985A396A3A7A3B0A7C0925F04D0929F
:106380006004E0926104F092620429813A814B81B9
:106390005C81C701B6010E946234A50194010E948C
:1063A0007A3760935B0470935C0480935D049093F0
:1063B0005E0420916C0430916D0440916E04509104
:1063C0006F04B8018DA99CA90E943C358111A1CA16
:1063D00020E030E0A901B8018DA99CA90E943F37B7
:1063E000181634F48091A50582608093A50507C036
:1063F00010928704109286040E94E8188ACAE596D3
:106400000FB6F894DEBF0FBECDBFDF91CF911F91C5
:106410000F91FF90EF90DF90CF90BF90AF909F9043
:106420008F907F906F905F904F903F902F90089546
:1064300087B1887F87B988B1876088B9ECE6F0E0DA
:10644000808187608083E8E6F0E0808182608083DD
:10645000089596B19095977041F0892F817091FDC4
:106460008260947019F08460089580E008951F920E
:106470000F920FB60F9211242F933F934F935F9378
:106480006F937F938F939F93AF93BF93EF93FF93FC
:106490000E942932882391F080FF03C00E948A164F
:1064A0000DC082FF04C080910101826005C081FFA0
:1064B00005C080910101886080930101FF91EF91F7
:1064C000BF91AF919F918F917F916F915F914F910C
:1064D0003F912F910F900FBE0F901F90189580E065
:1064E00008951F93CF93DF93EC0110E0BE01812F3D
:1064F0000E94D526811102C087E009C088818823C7
:1065000041F0CE010E946F1CCE010E944B050E94FB
:10651000C21F1F5F123051F7DF91CF911F91089575
:106520008F929F92AF92BF92CF92DF92EF92FF92A3
:106530001F93CF93DF93CDB7DEB729970FB6F894AB
:10654000DEBF0FBECDBF7C0181E08987F70181816D
:10655000833479F034F4882349F0843209F040C060
:1065600008C0873431F08835D9F503C00E94702007
:1065700035C0F7019281911138C18334A9F01CF420
:10658000843231F02BC0873461F08835F1F026C0B9
:106590008091A305887111F088E028C10E947420C1
:1065A0001DC00E94A5221AC08091A305823021F44B
:1065B0000E948A1685E006C08111EECF82E08093AA
:1065C000A30584E00E943D2009C08091A30581308D
:1065D00029F483E00E943D201092A30580E006C1CB
:1065E0009091A3059230C0F6893459F12CF483328E
:1065F00051F0883489F08AC08E3409F46AC082353B
:1066000009F440C083C082E08987F701828181114B
:10661000ECC00E941422E2CF8091C60684FFE3C042
:1066200084E08093A3050E94ED158091A20581115D
:10663000D5CF1092A3050E946829C7010E9471322C
:10664000CDCF82E08987F7018281811107C0C70120
:106650000E94F226C7010E948023C0CF8D3309F02B
:10666000C4C083E0F701E80FF11D9081DF011397AB
:106670009C938F5F90819111F5CF8987C7010E940C
:106680008825ACCFF7018281833509F0AEC08381C4
:10669000843509F0AAC084818D3309F0A6C08681B3
:1066A0008111A3C085E089878581843239F08A32DF
:1066B00039F0833209F099C082E003C081E001C063
:1066C0008FEF0E94A52588E00E943D200E948A1637
:1066D00085CF82E08987F7018281811113C010E0A4
:1066E000B701812F0E94D526811104C087E00E9446
:1066F000C21F04C0B701812F0E9466231F5F1230A2
:1067000079F76CCF911148CF11E001C010E0AE01D4
:106710004B5F5F4FBE01675F7F4FC7010E94A816A6
:10672000811102C082E062C0898521E0280F29879B
:10673000F701E80FF11D80818D3309F056C0112358
:1067400021F1822F90E0E22FF0E0D701AE0FBF1FC2
:106750003C91E81BF90BEE0DFF1D30832F5F3C9140
:106760003111F1CF2987C7010E944B0581113EC02D
:106770006D817E818F8198850E9448380E94B03556
:10678000862FB7010E947F2529CFAE014F5F5F4F53
:10679000BE01675F7F4FC7010E94A816882311F2D0
:1067A0008985F701E80FF11D808181111EC0CD8020
:1067B000DE80EF80F88420E030E04FE753E4C7014B
:1067C000B6010E943F37181684F089809A80AB800A
:1067D000BC80C701B6010E94B035862FB501A40167
:1067E0000E943C2703C085E001C083E029960FB6D4
:1067F000F894DEBF0FBECDBFDF91CF911F91FF9008
:10680000EF90DF90CF90BF90AF909F908F900895C2
:10681000CF93DF9324E0629FE00111248C0F9D1F32
:10682000FC0160817181828193810E94DE35CF57A6
:10683000D94F288139814A815B810E944335DF919C
:10684000CF910895FF920F931F93CF93DF938B0106
:10685000EC01F12C6F2DC8010E94083469937993E3
:1068600089939993F39483E0F812F4CFDF91CF9159
:106870001F910F91FF9008959FB7F8942091010107
:10688000822B809301019FBF08959FB7F8942091B8
:10689000010180958223809301019FBF08959FB7D6
:1068A000F89420910001822B809300019FBF0895EE
:1068B0009FB7F89420910001809582238093000176
:1068C0009FBF08955058BB27AA270ED076C23FD24B
:1068D00030F044D220F031F49F3F11F41EF40FC287
:1068E0000EF4E095E7FBDCC1E92F89D280F3BA17FB
:1068F000620773078407950718F071F49EF5B8C214
:106900000EF4E0950B2EBA2FA02D0B01B9019001CA
:106910000C01CA01A0011124FF27591B99F0593F0E
:1069200050F4503E68F11A16F040A22F232F342F56
:106930004427585FF3CF469537952795A795F040A4
:106940005395C9F77EF41F16BA0B620B730B840BB9
:10695000BAF09150A1F0FF0FBB1F661F771F881F71
:10696000C2F70EC0BA0F621F731F841F48F48795C9
:1069700077956795B795F7959E3F08F0B3CF9395B8
:10698000880F08F09927EE0F979587950895DFD126
:1069900058F080E891E009F49EEFE0D128F040E85B
:1069A00051E059F45EEF09C0AAC162C2E92FE07854
:1069B00026D268F3092E052AC1F3261737074807A0
:1069C000590738F00E2E07F8E02569F0E025E0645D
:1069D0000AC0EF6307F8009407FADB01B9019D01D3
:1069E000DC01CA01AD01EF935DD0E7D10AD05F9120
:1069F000552331F02BED3FE049E450FD49EC63CFE6
:106A00000895DF93DD27B92FBF7740E85FE31616BF
:106A1000170648075B0710F4D92F35D29F938F9341
:106A20007F936F9332D3EEE2F1E06CD1C6D12F9118
:106A30003F914F915F916AD2DD2349F09058A2EACD
:106A40002AED3FE049EC5FE3D0785D274DDFDF9131
:106A5000B4C1F7D180F09F3740F491110EF409C210
:106A600060E070E080E89FE3089526F01B16611D4A
:106A7000711D811D1BC135C1EFD008F481E008955F
:106A800075D1E395ABC10CD098C168D140F05FD10E
:106A900030F021F45F3F19F003C15111EAC12FC159
:106AA000AED198F39923C9F35523B1F3951B550B38
:106AB000BB27AA2762177307840738F09F5F5F4FD1
:106AC000220F331F441FAA1FA9F333D00E2E3AF012
:106AD000E0E830D091505040E695001CCAF729D02C
:106AE000FE2F27D0660F771F881FBB1F261737077B
:106AF0004807AB07B0E809F0BB0B802DBF01FF27AB
:106B000093585F4F2AF09E3F510568F0C9C0B1C14C
:106B10005F3FECF3983EDCF3869577956795B795E4
:106B2000F7959F5FC9F7880F911D9695879597F9FF
:106B30000895E1E0660F771F881FBB1F6217730778
:106B40008407BA0720F0621B730B840BBA0BEE1F8D
:106B500088F7E095089504D06894B1118AC108952A
:106B600056D188F09F5790F0B92F9927B751A0F0D0
:106B7000D1F0660F771F881F991F1AF0BA95C9F7D1
:106B800012C0B13081F074D1B1E0089571C1672FA6
:106B9000782F8827B85F39F0B93FCCF38695779581
:106BA0006795B395D9F73EF490958095709561956A
:106BB0007F4F8F4F9F4F0895E89409C097FB3EF495
:106BC00090958095709561957F4F8F4F9F4F99233A
:106BD000A9F0F92F96E9BB279395F69587957795B8
:106BE0006795B795F111F8CFFAF4BB0F11F460FF78
:106BF0001BC06F5F7F4F8F4F9F4F16C0882311F0D0
:106C000096E911C0772321F09EE8872F762F05C0E3
:106C1000662371F096E8862F70E060E02AF09A957E
:106C2000660F771F881FDAF7880F9695879597F973
:106C3000089507D180F09F3740F491110EF019C1EB
:106C400060E070E080E89FEB089526F41B16611D5C
:106C5000711D811D2BC045C0990F0008550FAA0B4F
:106C6000E0E8FEEF16161706E807F907C0F012165F
:106C70001306E407F50798F0621B730B840B950B62
:106C800039F40A2661F0232B242B252B21F40895B7
:106C90000A2609F4A140A6958FEF811D811D089554
:106CA00097F99F6780E870E060E00895882371F4A9
:106CB000772321F09850872B762F07C0662311F495
:106CC00099270DC09051862B70E060E02AF09A95CC
:106CD000660F771F881FDAF7880F9695879597F9C3
:106CE00008959F3F31F0915020F4879577956795EF
:106CF000B795880F911D9695879597F908959FEF01
:106D000080EC0895DF93CF931F930F93FF92EF9240
:106D1000DF927B018C01689405C0DA2EEF01F6D07A
:106D2000FE01E894A5912591359145915591AEF3D9
:106D3000EF01DADDFE019701A801DA9479F7DF901F
:106D4000EF90FF900F911F91CF91DF910895002454
:106D50000A941616170618060906089500240A94C0
:106D600012161306140605060895C9CF50D0E8F38D
:106D7000E894E0E0BB279F57F0F02AED3FE049ECB4
:106D800006C0EE0FBB0F661F771F881F28F0B23AB0
:106D900062077307840728F0B25A620B730B840BE7
:106DA000E3959A9572F7803830F49A95BB0F661F79
:106DB000771F881FD2F7904896CF092E0394000CB6
:106DC00011F4882352F0BB0F40F4BF2B11F460FF85
:106DD00004C06F5F7F4F8F4F9F4F0895EF93E0FF89
:106DE00006C0A2EA2AED3FE049EC5FEB7DDDE5DF7E
:106DF0000F90039401FC9058EBE5F1E057C157FD6B
:106E00009058440F551F59F05F3F71F04795880F18
:106E100097FB991F61F09F3F79F0879508951216AF
:106E200013061406551FF2CF4695F1DF08C016165B
:106E300017061806991FF1CF86957105610508940C
:106E40000895E5DFA0F0BEE7B91788F4BB279F38A7
:106E500060F41616B11D672F782F8827985FF7CF3B
:106E6000869577956795B11D93959639C8F30895E2
:106E7000E894BB2766277727CB0197F90895ECDEC6
:106E800008F48FEF08959B01AC0160E070E080E8AA
:106E90009FE3F9CDBCDF58F19E5758F19851A0F00F
:106EA000E9F0983020F5092E9927660F771F881F83
:106EB000991F0A94D1F712C0062E672F782F8827C2
:106EC000985F11F4000C07C0993FB4F3869577954D
:106ED00067959395D9F7611D711D811D3EF49095BD
:106EE0008095709561957F4F8F4F9F4F089568945F
:106EF000C0CFBECF0BD061CF2ADF28F02FDF18F034
:106F0000952309F0CDCEFBCE1124B3CF78DFA0F3CB
:106F1000959FD1F3950F50E0551F629FF001729F2E
:106F2000BB27F00DB11D639FAA27F00DB11DAA1F4D
:106F3000649F6627B00DA11D661F829F2227B00D9A
:106F4000A11D621F739FB00DA11D621F839FA00D25
:106F5000611D221F749F3327A00D611D231F849F75
:106F6000600D211D822F762F6A2F11249F575040CC
:106F70008AF0E1F088234AF0EE0FFF1FBB1F661F67
:106F8000771F881F91505040A9F79E3F510570F020
:106F900087CE6FCF5F3FECF3983EDCF38695779515
:106FA0006795B795F795E7959F5FC1F7FE2B880F1B
:106FB000911D9695879597F9089529DFE0F09E3702
:106FC000D8F09639B8F49E3848F4672F782F882780
:106FD000985FF9CF86957795679593959539D0F316
:106FE000B62FB1706B0F711D811D20F487957795B9
:106FF000679593955BCE75CE3CCF9F93B7DE0F9090
:1070000007FCEE5FEBCE11F40EF479CE6ACEFFDE14
:10701000D0F39923D9F3CEF39F57550B87FF3FD079
:107020000024A0E640EA900180585695979528F4F0
:10703000805C660F771F881F20F0261737074807E8
:1070400030F4621B730B840B202931294A2BA6953F
:1070500017940794202531254A2758F7660F771F84
:10706000881F20F026173707480730F4620B730B90
:10707000840B200D311D411DA09581F7B901842F8E
:107080009158880F9695879508959B01AC0132CF52
:10709000D8DE20F09F3708F4ECCE08CE22CE9150F7
:1070A0005040660F771F881FD2F708959F938F93E4
:1070B0007F936F93FF93EF939B01AC011BDFEF91E5
:1070C000FF9120DE2F913F914F915F9113CF991B3C
:1070D00079E004C0991F961708F0961B881F7A95CF
:1070E000C9F780950895A1E21A2EAA1BBB1BFD01CA
:1070F0000DC0AA1FBB1FEE1FFF1FA217B307E40797
:10710000F50720F0A21BB30BE40BF50B661F771FEE
:10711000881F991F1A9469F76095709580959095CE
:107120009B01AC01BD01CF010895EE0FFF1F05903B
:10713000F491E02D09940E94A638A59F900DB49F6C
:10714000900DA49F800D911D11240895A29FB00160
:10715000B39FC001A39F700D811D1124911DB29F8B
:0E716000700D811D1124911D0895F894FFCF2C
:00000001FF
